 nio

 Timestamp is ffffffff (Sun Feb  7 06:28:15 2106)

 Preferred load address is 10000000

 Start         Length     Name                   Class
 0001:00000000 000058faH .text$mn                CODE
 0002:00000000 000002a0H .idata$5                DATA
 0002:000002a0 00000004H .00cfg                  DATA
 0002:000002a4 00000004H .CRT$XCA                DATA
 0002:000002a8 00000004H .CRT$XCZ                DATA
 0002:000002ac 00000004H .CRT$XIA                DATA
 0002:000002b0 00000004H .CRT$XIZ                DATA
 0002:000002b4 00000004H .CRT$XPA                DATA
 0002:000002b8 00000004H .CRT$XPZ                DATA
 0002:000002bc 00000004H .CRT$XTA                DATA
 0002:000002c0 00000010H .CRT$XTZ                DATA
 0002:000002c4 00000000H .gfids$y                DATA
 0002:000002d0 000008e0H .rdata                  DATA
 0002:00000bb0 00000004H .rdata$sxdata           DATA
 0002:00000bb4 00000280H .rdata$zzzdbg           DATA
 0002:00000e34 00000004H .rtc$IAA                DATA
 0002:00000e38 00000004H .rtc$IZZ                DATA
 0002:00000e3c 00000004H .rtc$TAA                DATA
 0002:00000e40 00000008H .rtc$TZZ                DATA
 0002:00000e48 00000088H .xdata$x                DATA
 0002:00000ed0 00002b28H .edata                  DATA
 0002:000039f8 000000dcH .idata$2                DATA
 0002:00003ad4 00000014H .idata$3                DATA
 0002:00003ae8 000002a0H .idata$4                DATA
 0002:00003d88 00000c22H .idata$6                DATA
 0003:00000000 00000028H .data                   DATA
 0003:00000028 00000424H .bss                    DATA
 0004:00000000 00000060H .rsrc$01                DATA
 0004:00000060 00000300H .rsrc$02                DATA

  Address         Publics by Value              Rva+Base       Lib:Object

 0000:00000000       ___guard_iat_table         00000000     <absolute>
 0000:00000000       ___guard_fids_table        00000000     <absolute>
 0000:00000000       ___volatile_metadata       00000000     <absolute>
 0000:00000000       ___hybrid_auxiliary_iat    00000000     <absolute>
 0000:00000000       ___enclave_config          00000000     <absolute>
 0000:00000000       ___hybrid_code_map_count   00000000     <absolute>
 0000:00000000       ___guard_longjmp_table     00000000     <absolute>
 0000:00000000       ___hybrid_code_map         00000000     <absolute>
 0000:00000000       ___guard_fids_count        00000000     <absolute>
 0000:00000000       ___dynamic_value_reloc_table 00000000     <absolute>
 0000:00000000       ___guard_iat_count         00000000     <absolute>
 0000:00000000       ___guard_longjmp_count     00000000     <absolute>
 0000:00000001       ___safe_se_handler_count   00000001     <absolute>
 0000:00000100       ___guard_flags             00000100     <absolute>
 0000:00000000       ___ImageBase               10000000     <linker-defined>
 0001:00000000       _Java_sun_nio_ch_DatagramChannelImpl_disconnect0@16 10001000 f   DatagramChannelImpl.obj
 0001:00000087       _Java_sun_nio_ch_DatagramChannelImpl_initIDs@8 10001087 f   DatagramChannelImpl.obj
 0001:00000144       _Java_sun_nio_ch_DatagramChannelImpl_receive0@28 10001144 f   DatagramChannelImpl.obj
 0001:000002ec       _Java_sun_nio_ch_DatagramChannelImpl_send0@36 100012ec f   DatagramChannelImpl.obj
 0001:00000397       _purgeOutstandingICMP      10001397 f   DatagramChannelImpl.obj
 0001:0000045c       _Java_sun_nio_ch_DatagramDispatcher_read0@24 1000145c f   DatagramDispatcher.obj
 0001:00000504       _Java_sun_nio_ch_DatagramDispatcher_readv0@24 10001504 f   DatagramDispatcher.obj
 0001:00000608       _Java_sun_nio_ch_DatagramDispatcher_write0@24 10001608 f   DatagramDispatcher.obj
 0001:000006a2       _Java_sun_nio_ch_DatagramDispatcher_writev0@24 100016a2 f   DatagramDispatcher.obj
 0001:00000795       _Java_sun_nio_ch_FileChannelImpl_initIDs@8 10001795 f   FileChannelImpl.obj
 0001:000007cf       _Java_sun_nio_ch_FileChannelImpl_map0@28 100017cf f   FileChannelImpl.obj
 0001:0000089b       _Java_sun_nio_ch_FileChannelImpl_transferTo0@32 1000189b f   FileChannelImpl.obj
 0001:0000095c       _Java_sun_nio_ch_FileChannelImpl_unmap0@24 1000195c f   FileChannelImpl.obj
 0001:00000982       _Java_sun_nio_ch_FileDispatcherImpl_close0@12 10001982 f   FileDispatcherImpl.obj
 0001:000009b2       _Java_sun_nio_ch_FileDispatcherImpl_duplicateHandle@16 100019b2 f   FileDispatcherImpl.obj
 0001:000009ea       _Java_sun_nio_ch_FileDispatcherImpl_force0@16 100019ea f   FileDispatcherImpl.obj
 0001:00000a2c       _Java_sun_nio_ch_FileDispatcherImpl_lock0@36 10001a2c f   FileDispatcherImpl.obj
 0001:00000acd       _Java_sun_nio_ch_FileDispatcherImpl_pread0@32 10001acd f   FileDispatcherImpl.obj
 0001:00000bc2       _Java_sun_nio_ch_FileDispatcherImpl_pwrite0@32 10001bc2 f   FileDispatcherImpl.obj
 0001:00000c8b       _Java_sun_nio_ch_FileDispatcherImpl_read0@24 10001c8b f   FileDispatcherImpl.obj
 0001:00000d04       _Java_sun_nio_ch_FileDispatcherImpl_readv0@24 10001d04 f   FileDispatcherImpl.obj
 0001:00000dda       _Java_sun_nio_ch_FileDispatcherImpl_release0@28 10001dda f   FileDispatcherImpl.obj
 0001:00000e58       _Java_sun_nio_ch_FileDispatcherImpl_seek0@20 10001e58 f   FileDispatcherImpl.obj
 0001:00000ec6       _Java_sun_nio_ch_FileDispatcherImpl_setDirect0@16 10001ec6 f   FileDispatcherImpl.obj
 0001:00000f2e       _Java_sun_nio_ch_FileDispatcherImpl_size0@12 10001f2e f   FileDispatcherImpl.obj
 0001:00000f6e       _Java_sun_nio_ch_FileDispatcherImpl_truncate0@20 10001f6e f   FileDispatcherImpl.obj
 0001:00000fb7       _Java_sun_nio_ch_FileDispatcherImpl_write0@28 10001fb7 f   FileDispatcherImpl.obj
 0001:00001038       _Java_sun_nio_ch_FileDispatcherImpl_writev0@28 10002038 f   FileDispatcherImpl.obj
 0001:00001113       _Java_sun_nio_ch_FileKey_init@12 10002113 f   FileKey.obj
 0001:000011a2       _Java_sun_nio_ch_FileKey_initIDs@8 100021a2 f   FileKey.obj
 0001:00001202       _Java_sun_nio_ch_IOUtil_configureBlocking@16 10002202 f   IOUtil.obj
 0001:0000125d       _Java_sun_nio_ch_IOUtil_drain@12 1000225d f   IOUtil.obj
 0001:000012f9       _Java_sun_nio_ch_IOUtil_fdVal@12 100022f9 f   IOUtil.obj
 0001:0000130b       _Java_sun_nio_ch_IOUtil_initIDs@8 1000230b f   IOUtil.obj
 0001:0000135d       _Java_sun_nio_ch_IOUtil_iovMax@8 1000235d f   IOUtil.obj
 0001:0000135d       _Java_sun_nio_ch_Net_polloutValue@8 1000235d f   Net.obj
 0001:00001363       _Java_sun_nio_ch_IOUtil_randomBytes@12 10002363 f   IOUtil.obj
 0001:00001368       _Java_sun_nio_ch_IOUtil_setfdVal@16 10002368 f   IOUtil.obj
 0001:00001386       _convertLongReturnVal      10002386 f   IOUtil.obj
 0001:000013c5       _convertReturnVal          100023c5 f   IOUtil.obj
 0001:000013ec       _fdval                     100023ec f   IOUtil.obj
 0001:00001404       _handleval                 10002404 f   IOUtil.obj
 0001:0000141c       _Java_sun_nio_fs_WindowsNativeDispatcher_CloseHandle@16 1000241c f   WindowsNativeDispatcher.obj
 0001:0000141c       _Java_sun_nio_ch_Iocp_close0@16 1000241c f   Iocp.obj
 0001:00001429       _Java_sun_nio_ch_Iocp_createIoCompletionPort@32 10002429 f   Iocp.obj
 0001:0000145a       _Java_sun_nio_ch_Iocp_getErrorMessage@12 1000245a f   Iocp.obj
 0001:0000145a       _Java_sun_nio_fs_WindowsNativeDispatcher_FormatMessage@12 1000245a f   WindowsNativeDispatcher.obj
 0001:000014c4       _Java_sun_nio_ch_Iocp_getQueuedCompletionStatus@20 100024c4 f   Iocp.obj
 0001:00001563       _Java_sun_nio_ch_Iocp_initIDs@8 10002563 f   Iocp.obj
 0001:000015ea       _Java_sun_nio_ch_Iocp_postQueuedCompletionStatus@20 100025ea f   Iocp.obj
 0001:00001611       _Java_java_nio_MappedByteBuffer_force0@28 10002611 f   MappedByteBuffer.obj
 0001:000016a7       _Java_java_nio_MappedByteBuffer_isLoaded0@28 100026a7 f   MappedByteBuffer.obj
 0001:000016ac       _Java_java_nio_MappedByteBuffer_load0@24 100026ac f   MappedByteBuffer.obj
 0001:000016af       _IN6_IS_ADDR_LOOPBACK      100026af f i Net.obj
 0001:000016ec       _Java_sun_nio_ch_Net_bind0@28 100026ec f   Net.obj
 0001:00001764       _Java_sun_nio_ch_Net_blockOrUnblock4@28 10002764 f   Net.obj
 0001:00001808       _Java_sun_nio_ch_Net_blockOrUnblock6@28 10002808 f   Net.obj
 0001:0000184a       _Java_sun_nio_ch_Net_canIPv6SocketJoinIPv4Group0@8 1000284a f   Net.obj
 0001:0000184a       _Java_sun_nio_ch_Net_canJoin6WithIPv4Group0@8 1000284a f   Net.obj
 0001:0000184a       _Java_sun_nio_ch_Net_isReusePortAvailable0@8 1000284a f   Net.obj
 0001:0000184f       _Java_sun_nio_ch_Net_connect0@24 1000284f f   Net.obj
 0001:000019a4       _Java_sun_nio_ch_Net_getIntOption0@24 100029a4 f   Net.obj
 0001:00001a6b       _Java_sun_nio_ch_Net_getInterface4@12 10002a6b f   Net.obj
 0001:00001abe       _Java_sun_nio_ch_Net_getInterface6@12 10002abe f   Net.obj
 0001:00001b0c       _Java_sun_nio_ch_Net_initIDs@8 10002b0c f   Net.obj
 0001:00001b18       _Java_sun_nio_ch_Net_pollerrValue@8 10002b18 f   Net.obj
 0001:00001b18       _Java_sun_nio_ch_Net_isExclusiveBindAvailable@8 10002b18 f   Net.obj
 0001:00001b1e       _Java_sun_nio_ch_Net_isIPv6Available0@8 10002b1e f   Net.obj
 0001:00001b2b       _Java_sun_nio_ch_Net_joinOrDrop4@28 10002b2b f   Net.obj
 0001:00001bfc       _Java_sun_nio_ch_Net_joinOrDrop6@28 10002bfc f   Net.obj
 0001:00001c9d       _Java_sun_nio_ch_Net_listen@16 10002c9d f   Net.obj
 0001:00001c9d       _Java_sun_nio_ch_ServerSocketChannelImpl_listen@16 10002c9d f   ServerSocketChannelImpl.obj
 0001:00001cd4       _Java_sun_nio_ch_Net_localInetAddress@12 10002cd4 f   Net.obj
 0001:00001d41       _Java_sun_nio_ch_Net_localPort@12 10002d41 f   Net.obj
 0001:00001db5       _Java_sun_nio_ch_Net_poll@24 10002db5 f   Net.obj
 0001:00001eff       _Java_sun_nio_ch_Net_pollconnValue@8 10002eff f   Net.obj
 0001:00001f07       _Java_sun_nio_ch_Net_pollhupValue@8 10002f07 f   Net.obj
 0001:00001f0d       _Java_sun_nio_ch_Net_pollinValue@8 10002f0d f   Net.obj
 0001:00001f15       _Java_sun_nio_ch_Net_pollnvalValue@8 10002f15 f   Net.obj
 0001:00001f1b       _Java_sun_nio_ch_Net_remoteInetAddress@12 10002f1b f   Net.obj
 0001:00001f88       _Java_sun_nio_ch_Net_remotePort@12 10002f88 f   Net.obj
 0001:00001ffc       _Java_sun_nio_ch_Net_setIntOption0@32 10002ffc f   Net.obj
 0001:00002084       _Java_sun_nio_ch_Net_setInterface4@16 10003084 f   Net.obj
 0001:000020ca       _Java_sun_nio_ch_Net_setInterface6@16 100030ca f   Net.obj
 0001:00002105       _Java_sun_nio_ch_Net_shutdown@16 10003105 f   Net.obj
 0001:0000214c       _Java_sun_nio_ch_Net_socket0@24 1000314c f   Net.obj
 0001:000022df       _Java_sun_nio_fs_RegistryFileTypeDetector_queryStringValue@24 100032df f   RegistryFileTypeDetector.obj
 0001:000023a5       _Java_sun_nio_ch_ServerSocketChannelImpl_accept0@20 100033a5 f   ServerSocketChannelImpl.obj
 0001:0000249c       _Java_sun_nio_ch_ServerSocketChannelImpl_initIDs@8 1000349c f   ServerSocketChannelImpl.obj
 0001:00002516       _Java_sun_nio_ch_SocketChannelImpl_checkConnect@16 10003516 f   SocketChannelImpl.obj
 0001:00002659       _Java_sun_nio_ch_SocketChannelImpl_initIDs@8 10003659 f   SocketChannelImpl.obj
 0001:0000268a       _Java_sun_nio_ch_SocketChannelImpl_sendOutOfBandData@16 1000368a f   SocketChannelImpl.obj
 0001:000026c6       _handleSocketError         100036c6 f   SocketChannelImpl.obj
 0001:000026d9       _Java_sun_nio_ch_SocketDispatcher_close0@12 100036d9 f   SocketDispatcher.obj
 0001:00002705       _Java_sun_nio_ch_SocketDispatcher_preClose0@12 10003705 f   SocketDispatcher.obj
 0001:00002750       _Java_sun_nio_ch_SocketDispatcher_read0@24 10003750 f   SocketDispatcher.obj
 0001:000027d5       _Java_sun_nio_ch_SocketDispatcher_readv0@24 100037d5 f   SocketDispatcher.obj
 0001:000028dd       _Java_sun_nio_ch_SocketDispatcher_write0@24 100038dd f   SocketDispatcher.obj
 0001:00002988       _Java_sun_nio_ch_SocketDispatcher_writev0@24 10003988 f   SocketDispatcher.obj
 0001:00002b17       _Java_sun_nio_ch_WindowsAsynchronousFileChannelImpl_lockFile@44 10003b17 f   WindowsAsynchronousFileChannelImpl.obj
 0001:00002b79       _Java_sun_nio_ch_WindowsAsynchronousFileChannelImpl_readFile@44 10003b79 f   WindowsAsynchronousFileChannelImpl.obj
 0001:00002bd4       _Java_sun_nio_ch_WindowsAsynchronousFileChannelImpl_writeFile@44 10003bd4 f   WindowsAsynchronousFileChannelImpl.obj
 0001:00002c25       _Java_sun_nio_ch_WindowsAsynchronousServerSocketChannelImpl_accept0@40 10003c25 f   WindowsAsynchronousServerSocketChannelImpl.obj
 0001:00002c85       _Java_sun_nio_ch_WindowsAsynchronousServerSocketChannelImpl_closesocket0@16 10003c85 f   WindowsAsynchronousServerSocketChannelImpl.obj
 0001:00002c85       _Java_sun_nio_ch_WindowsAsynchronousSocketChannelImpl_closesocket0@16 10003c85 f   WindowsAsynchronousSocketChannelImpl.obj
 0001:00002ca5       _Java_sun_nio_ch_WindowsAsynchronousServerSocketChannelImpl_initIDs@8 10003ca5 f   WindowsAsynchronousServerSocketChannelImpl.obj
 0001:00002d3e       _Java_sun_nio_ch_WindowsAsynchronousServerSocketChannelImpl_updateAcceptContext@24 10003d3e f   WindowsAsynchronousServerSocketChannelImpl.obj
 0001:00002d64       _Java_sun_nio_ch_WindowsAsynchronousSocketChannelImpl_connect0@36 10003d64 f   WindowsAsynchronousSocketChannelImpl.obj
 0001:00002dfe       _Java_sun_nio_ch_WindowsAsynchronousSocketChannelImpl_initIDs@8 10003dfe f   WindowsAsynchronousSocketChannelImpl.obj
 0001:00002e96       _Java_sun_nio_ch_WindowsAsynchronousSocketChannelImpl_read0@36 10003e96 f   WindowsAsynchronousSocketChannelImpl.obj
 0001:00002efd       _Java_sun_nio_ch_WindowsAsynchronousSocketChannelImpl_shutdown0@20 10003efd f   WindowsAsynchronousSocketChannelImpl.obj
 0001:00002f21       _Java_sun_nio_ch_WindowsAsynchronousSocketChannelImpl_updateConnectContext@16 10003f21 f   WindowsAsynchronousSocketChannelImpl.obj
 0001:00002f3c       _Java_sun_nio_ch_WindowsAsynchronousSocketChannelImpl_write0@36 10003f3c f   WindowsAsynchronousSocketChannelImpl.obj
 0001:00002f9c       _Java_sun_nio_fs_WindowsNativeDispatcher_AccessCheck@44 10003f9c f   WindowsNativeDispatcher.obj
 0001:00003073       _Java_sun_nio_fs_WindowsNativeDispatcher_AddAccessAllowedAceEx@32 10004073 f   WindowsNativeDispatcher.obj
 0001:000030a3       _Java_sun_nio_fs_WindowsNativeDispatcher_AddAccessDeniedAceEx@32 100040a3 f   WindowsNativeDispatcher.obj
 0001:000030d3       _Java_sun_nio_fs_WindowsNativeDispatcher_AdjustTokenPrivileges@28 100040d3 f   WindowsNativeDispatcher.obj
 0001:0000313f       _Java_sun_nio_fs_WindowsNativeDispatcher_CancelIo@16 1000413f f   WindowsNativeDispatcher.obj
 0001:00003162       _Java_sun_nio_fs_WindowsNativeDispatcher_ConvertSidToStringSid@16 10004162 f   WindowsNativeDispatcher.obj
 0001:000031ba       _Java_sun_nio_fs_WindowsNativeDispatcher_ConvertStringSidToSid0@16 100041ba f   WindowsNativeDispatcher.obj
 0001:000031e7       _Java_sun_nio_fs_WindowsNativeDispatcher_CopyFileEx0@36 100041e7 f   WindowsNativeDispatcher.obj
 0001:00003219       _Java_sun_nio_fs_WindowsNativeDispatcher_CreateDirectory0@24 10004219 f   WindowsNativeDispatcher.obj
 0001:0000325a       _Java_sun_nio_fs_WindowsNativeDispatcher_CreateEvent@16 1000425a f   WindowsNativeDispatcher.obj
 0001:00003290       _Java_sun_nio_fs_WindowsNativeDispatcher_CreateFile0@40 10004290 f   WindowsNativeDispatcher.obj
 0001:000032e7       _Java_sun_nio_fs_WindowsNativeDispatcher_CreateHardLink0@24 100042e7 f   WindowsNativeDispatcher.obj
 0001:00003310       _Java_sun_nio_fs_WindowsNativeDispatcher_CreateIoCompletionPort@32 10004310 f   WindowsNativeDispatcher.obj
 0001:00003344       _Java_sun_nio_fs_WindowsNativeDispatcher_CreateSymbolicLink0@28 10004344 f   WindowsNativeDispatcher.obj
 0001:0000336f       _Java_sun_nio_fs_WindowsNativeDispatcher_DeleteFile0@16 1000436f f   WindowsNativeDispatcher.obj
 0001:00003392       _Java_sun_nio_fs_WindowsNativeDispatcher_DeviceIoControlGetReparsePoint@28 10004392 f   WindowsNativeDispatcher.obj
 0001:000033cc       _Java_sun_nio_fs_WindowsNativeDispatcher_DeviceIoControlSetSparse@16 100043cc f   WindowsNativeDispatcher.obj
 0001:00003402       _Java_sun_nio_fs_WindowsNativeDispatcher_DuplicateTokenEx@20 10004402 f   WindowsNativeDispatcher.obj
 0001:00003439       _Java_sun_nio_fs_WindowsNativeDispatcher_FindClose@16 10004439 f   WindowsNativeDispatcher.obj
 0001:0000345c       _Java_sun_nio_fs_WindowsNativeDispatcher_FindFirstFile0@20 1000445c f   WindowsNativeDispatcher.obj
 0001:00003523       _Java_sun_nio_fs_WindowsNativeDispatcher_FindFirstFile1@24 10004523 f   WindowsNativeDispatcher.obj
 0001:00003552       _Java_sun_nio_fs_WindowsNativeDispatcher_FindFirstStream0@20 10004552 f   WindowsNativeDispatcher.obj
 0001:00003628       _Java_sun_nio_fs_WindowsNativeDispatcher_FindNextFile@24 10004628 f   WindowsNativeDispatcher.obj
 0001:0000367d       _Java_sun_nio_fs_WindowsNativeDispatcher_FindNextStream@16 1000467d f   WindowsNativeDispatcher.obj
 0001:000036f5       _Java_sun_nio_fs_WindowsNativeDispatcher_GetAce@20 100046f5 f   WindowsNativeDispatcher.obj
 0001:0000372c       _Java_sun_nio_fs_WindowsNativeDispatcher_GetAclInformation0@20 1000472c f   WindowsNativeDispatcher.obj
 0001:00003794       _Java_sun_nio_fs_WindowsNativeDispatcher_GetCurrentProcess@8 10004794 f   WindowsNativeDispatcher.obj
 0001:0000379e       _Java_sun_nio_fs_WindowsNativeDispatcher_GetCurrentThread@8 1000479e f   WindowsNativeDispatcher.obj
 0001:000037a8       _Java_sun_nio_fs_WindowsNativeDispatcher_GetDiskFreeSpace0@20 100047a8 f   WindowsNativeDispatcher.obj
 0001:000037fc       _Java_sun_nio_fs_WindowsNativeDispatcher_GetDiskFreeSpaceEx0@20 100047fc f   WindowsNativeDispatcher.obj
 0001:0000387f       _Java_sun_nio_fs_WindowsNativeDispatcher_GetDriveType0@16 1000487f f   WindowsNativeDispatcher.obj
 0001:0000388c       _Java_sun_nio_fs_WindowsNativeDispatcher_GetFileAttributes0@16 1000488c f   WindowsNativeDispatcher.obj
 0001:000038b6       _Java_sun_nio_fs_WindowsNativeDispatcher_GetFileAttributesEx0@24 100048b6 f   WindowsNativeDispatcher.obj
 0001:000038df       _Java_sun_nio_fs_WindowsNativeDispatcher_GetFileInformationByHandle@24 100048df f   WindowsNativeDispatcher.obj
 0001:00003906       _Java_sun_nio_fs_WindowsNativeDispatcher_GetFileSecurity0@32 10004906 f   WindowsNativeDispatcher.obj
 0001:00003954       _Java_sun_nio_fs_WindowsNativeDispatcher_GetFinalPathNameByHandle@16 10004954 f   WindowsNativeDispatcher.obj
 0001:00003a2f       _Java_sun_nio_fs_WindowsNativeDispatcher_GetFullPathName0@16 10004a2f f   WindowsNativeDispatcher.obj
 0001:00003b0a       _Java_sun_nio_fs_WindowsNativeDispatcher_GetLengthSid@16 10004b0a f   WindowsNativeDispatcher.obj
 0001:00003b17       _Java_sun_nio_fs_WindowsNativeDispatcher_GetLogicalDrives@8 10004b17 f   WindowsNativeDispatcher.obj
 0001:00003b3c       _Java_sun_nio_fs_WindowsNativeDispatcher_GetOverlappedResult@24 10004b3c f   WindowsNativeDispatcher.obj
 0001:00003b72       _Java_sun_nio_fs_WindowsNativeDispatcher_GetQueuedCompletionStatus0@20 10004b72 f   WindowsNativeDispatcher.obj
 0001:00003bff       _Java_sun_nio_fs_WindowsNativeDispatcher_GetSecurityDescriptorDacl@16 10004bff f   WindowsNativeDispatcher.obj
 0001:00003c53       _Java_sun_nio_fs_WindowsNativeDispatcher_GetSecurityDescriptorOwner@16 10004c53 f   WindowsNativeDispatcher.obj
 0001:00003c86       _Java_sun_nio_fs_WindowsNativeDispatcher_GetTokenInformation@32 10004c86 f   WindowsNativeDispatcher.obj
 0001:00003cd0       _Java_sun_nio_fs_WindowsNativeDispatcher_GetVolumeInformation0@20 10004cd0 f   WindowsNativeDispatcher.obj
 0001:00003de8       _Java_sun_nio_fs_WindowsNativeDispatcher_GetVolumePathName0@16 10004de8 f   WindowsNativeDispatcher.obj
 0001:00003e5c       _Java_sun_nio_fs_WindowsNativeDispatcher_InitializeAcl@20 10004e5c f   WindowsNativeDispatcher.obj
 0001:00003e85       _Java_sun_nio_fs_WindowsNativeDispatcher_InitializeSecurityDescriptor@16 10004e85 f   WindowsNativeDispatcher.obj
 0001:00003eaa       _Java_sun_nio_fs_WindowsNativeDispatcher_LocalFree@16 10004eaa f   WindowsNativeDispatcher.obj
 0001:00003eb7       _Java_sun_nio_fs_WindowsNativeDispatcher_LookupAccountName0@28 10004eb7 f   WindowsNativeDispatcher.obj
 0001:00003f43       _Java_sun_nio_fs_WindowsNativeDispatcher_LookupAccountSid0@20 10004f43 f   WindowsNativeDispatcher.obj
 0001:0000404b       _Java_sun_nio_fs_WindowsNativeDispatcher_LookupPrivilegeValue0@16 1000504b f   WindowsNativeDispatcher.obj
 0001:00004096       _Java_sun_nio_fs_WindowsNativeDispatcher_MoveFileEx0@28 10005096 f   WindowsNativeDispatcher.obj
 0001:000040c1       _Java_sun_nio_fs_WindowsNativeDispatcher_OpenProcessToken@20 100050c1 f   WindowsNativeDispatcher.obj
 0001:000040f2       _Java_sun_nio_fs_WindowsNativeDispatcher_OpenThreadToken@24 100050f2 f   WindowsNativeDispatcher.obj
 0001:00004140       _Java_sun_nio_fs_WindowsNativeDispatcher_PostQueuedCompletionStatus@24 10005140 f   WindowsNativeDispatcher.obj
 0001:0000416b       _Java_sun_nio_fs_WindowsNativeDispatcher_ReadDirectoryChangesW@52 1000516b f   WindowsNativeDispatcher.obj
 0001:000041ab       _Java_sun_nio_fs_WindowsNativeDispatcher_RemoveDirectory0@16 100051ab f   WindowsNativeDispatcher.obj
 0001:000041ce       _Java_sun_nio_fs_WindowsNativeDispatcher_SetEndOfFile@16 100051ce f   WindowsNativeDispatcher.obj
 0001:000041f1       _Java_sun_nio_fs_WindowsNativeDispatcher_SetFileAttributes0@20 100051f1 f   WindowsNativeDispatcher.obj
 0001:00004218       _Java_sun_nio_fs_WindowsNativeDispatcher_SetFileSecurity0@28 10005218 f   WindowsNativeDispatcher.obj
 0001:00004243       _Java_sun_nio_fs_WindowsNativeDispatcher_SetFileTime@40 10005243 f   WindowsNativeDispatcher.obj
 0001:0000429d       _Java_sun_nio_fs_WindowsNativeDispatcher_SetSecurityDescriptorDacl@24 1000529d f   WindowsNativeDispatcher.obj
 0001:000042c8       _Java_sun_nio_fs_WindowsNativeDispatcher_SetSecurityDescriptorOwner@24 100052c8 f   WindowsNativeDispatcher.obj
 0001:000042f1       _Java_sun_nio_fs_WindowsNativeDispatcher_SetThreadToken@24 100052f1 f   WindowsNativeDispatcher.obj
 0001:00004318       _Java_sun_nio_fs_WindowsNativeDispatcher_initIDs@8 10005318 f   WindowsNativeDispatcher.obj
 0001:0000462b       _Java_sun_nio_ch_WindowsSelectorImpl_00024SubSelector_poll0@48 1000562b f   WindowsSelectorImpl.obj
 0001:000048c9       _Java_sun_nio_ch_WindowsSelectorImpl_discardUrgentData@12 100058c9 f   WindowsSelectorImpl.obj
 0001:00004906       _Java_sun_nio_ch_WindowsSelectorImpl_resetWakeupSocket0@12 10005906 f   WindowsSelectorImpl.obj
 0001:00004989       _Java_sun_nio_ch_WindowsSelectorImpl_setWakeupSocket0@12 10005989 f   WindowsSelectorImpl.obj
 0001:000049a6       _JNI_OnLoad@8              100059a6 f   nio_util.obj
 0001:000049cd       ___WSAFDIsSet@8            100059cd f   ws2_32:WS2_32.dll
 0001:000049d3       _JNU_ThrowByName@12        100059d3 f   java:java.dll
 0001:000049d9       _JNU_ThrowOutOfMemoryError@8 100059d9 f   java:java.dll
 0001:000049df       _JNU_ThrowIOExceptionWithLastError@8 100059df f   java:java.dll
 0001:000049e5       _Java_sun_security_provider_NativeSeedGenerator_nativeGenerateSeed@12 100059e5 f   java:java.dll
 0001:000049eb       _JNU_ThrowInternalError@8  100059eb f   java:java.dll
 0001:000049f1       _JNU_NewObjectByName       100059f1 f   java:java.dll
 0001:000049f7       _NET_InetAddressToSockaddr@24 100059f7 f   net:net.dll
 0001:000049fd       _NET_SockaddrToInetAddress@12 100059fd f   net:net.dll
 0001:00004a03       _NET_GetPortFromSockaddr@4 10005a03 f   net:net.dll
 0001:00004a09       _NET_SockaddrEqualsInetAddress@12 10005a09 f   net:net.dll
 0001:00004a0f       _NET_WinBind@16            10005a0f f   net:net.dll
 0001:00004a15       _NET_EnableFastTcpLoopbackConnect@4 10005a15 f   net:net.dll
 0001:00004a1b       _initInetAddressIDs@4      10005a1b f   net:net.dll
 0001:00004a21       _NET_ThrowNew@12           10005a21 f   net:net.dll
 0001:00004a27       _ipv6_available@0          10005a27 f   net:net.dll
 0001:00004a2d       _NET_GetSockOpt@20         10005a2d f   net:net.dll
 0001:00004a33       _NET_SetSockOpt@20         10005a33 f   net:net.dll
 0001:00004a39       _NET_EnableFastTcpLoopback@4 10005a39 f   net:net.dll
 0001:00004a3f       _ConvertSidToStringSidW@8  10005a3f f   advapi32:ADVAPI32.dll
 0001:00004a45       _ConvertStringSidToSidW@8  10005a45 f   advapi32:ADVAPI32.dll
 0001:00004a4b       @__security_check_cookie@4 10005a4b f   MSVCRT:secchk.obj
 0001:00004a60       __alldvrm                  10005a60 f   MSVCRT:lldvrm.obj
 0001:00004b40       __alldiv                   10005b40 f   MSVCRT:lldiv.obj
 0001:00004bf0       __allrem                   10005bf0 f   MSVCRT:llrem.obj
 0001:00004fc2       __DllMainCRTStartup@12     10005fc2 f   MSVCRT:dll_dllmain.obj
 0001:00004fe5       ___raise_securityfailure   10005fe5 f   MSVCRT:gs_report.obj
 0001:0000500d       ___report_gsfailure        1000600d f   MSVCRT:gs_report.obj
 0001:00005153       ___security_init_cookie    10006153 f   MSVCRT:gs_support.obj
 0001:0000519e       _DllMain@12                1000619e f   MSVCRT:dll_dllmain_stub.obj
 0001:000051c0       ?__scrt_initialize_type_info@@YAXXZ 100061c0 f   MSVCRT:tncleanup.obj
 0001:000051cc       ?__scrt_uninitialize_type_info@@YAXXZ 100061cc f   MSVCRT:tncleanup.obj
 0001:000051d8       ___local_stdio_printf_options 100061d8 f i MSVCRT:default_local_stdio_options.obj
 0001:000051de       ___local_stdio_scanf_options 100061de f i MSVCRT:default_local_stdio_options.obj
 0001:000051e4       ___scrt_initialize_default_local_stdio_options 100061e4 f   MSVCRT:default_local_stdio_options.obj
 0001:00005245       ___scrt_acquire_startup_lock 10006245 f   MSVCRT:utility.obj
 0001:00005277       ___scrt_dllmain_after_initialize_c 10006277 f   MSVCRT:utility.obj
 0001:000052a2       ___scrt_dllmain_before_initialize_c 100062a2 f   MSVCRT:utility.obj
 0001:000052b0       ___scrt_dllmain_crt_thread_attach 100062b0 f   MSVCRT:utility.obj
 0001:000052cf       ___scrt_dllmain_crt_thread_detach 100062cf f   MSVCRT:utility.obj
 0001:000052dc       ___scrt_dllmain_exception_filter 100062dc f   MSVCRT:utility.obj
 0001:00005310       ___scrt_dllmain_uninitialize_c 10006310 f   MSVCRT:utility.obj
 0001:00005333       ___scrt_dllmain_uninitialize_critical 10006333 f   MSVCRT:utility.obj
 0001:00005340       ___scrt_initialize_crt     10006340 f   MSVCRT:utility.obj
 0001:00005379       ___scrt_initialize_onexit_tables 10006379 f   MSVCRT:utility.obj
 0001:0000541e       ___scrt_is_nonwritable_in_current_image 1000641e f   MSVCRT:utility.obj
 0001:000054b2       ___scrt_release_startup_lock 100064b2 f   MSVCRT:utility.obj
 0001:000054cf       ___scrt_uninitialize_crt   100064cf f   MSVCRT:utility.obj
 0001:000054f7       ___scrt_get_dyn_tls_init_callback 100064f7 f   MSVCRT:dyn_tls_init.obj
 0001:000054fd       ___scrt_fastfail           100064fd f   MSVCRT:utility_desktop.obj
 0001:00005617       __crt_debugger_hook        10006617 f   MSVCRT:utility_desktop.obj
 0001:0000561f       __RTC_Initialize           1000661f f   MSVCRT:initsect.obj
 0001:0000564b       __RTC_Terminate            1000664b f   MSVCRT:initsect.obj
 0001:00005680       __SEH_prolog4              10006680 f   MSVCRT:sehprolg4.obj
 0001:000056c6       __SEH_epilog4              100066c6 f   MSVCRT:sehprolg4.obj
 0001:000056db       __except_handler4          100066db f   MSVCRT:chandler4gs.obj
 0001:000056fe       @_guard_check_icall_nop@4  100066fe f i MSVCRT:guard_support.obj
 0001:000056ff       ___isa_available_init      100066ff f   MSVCRT:cpu_disp.obj
 0001:00005896       __get_startup_argv_mode    10006896 f   MSVCRT:argv_mode.obj
 0001:0000589a       ___scrt_is_ucrt_dll_in_use 1000689a f   MSVCRT:ucrt_detection.obj
 0001:000058a6       _TransmitFile@28           100068a6 f   Mswsock:MSWSOCK.dll
 0001:000058ac       _IsProcessorFeaturePresent@4 100068ac f   kernel32:KERNEL32.dll
 0001:000058b2       _memset                    100068b2 f   vcruntime:VCRUNTIME140.dll
 0001:000058b8       ___std_type_info_destroy_list 100068b8 f   vcruntime:VCRUNTIME140.dll
 0001:000058be       __except_handler4_common   100068be f   vcruntime:VCRUNTIME140.dll
 0001:000058c4       __initterm                 100068c4 f   ucrt:api-ms-win-crt-runtime-l1-1-0.dll
 0001:000058ca       __initterm_e               100068ca f   ucrt:api-ms-win-crt-runtime-l1-1-0.dll
 0001:000058d0       __seh_filter_dll           100068d0 f   ucrt:api-ms-win-crt-runtime-l1-1-0.dll
 0001:000058d6       __configure_narrow_argv    100068d6 f   ucrt:api-ms-win-crt-runtime-l1-1-0.dll
 0001:000058dc       __initialize_narrow_environment 100068dc f   ucrt:api-ms-win-crt-runtime-l1-1-0.dll
 0001:000058e2       __initialize_onexit_table  100068e2 f   ucrt:api-ms-win-crt-runtime-l1-1-0.dll
 0001:000058e8       __execute_onexit_table     100068e8 f   ucrt:api-ms-win-crt-runtime-l1-1-0.dll
 0001:000058ee       __cexit                    100068ee f   ucrt:api-ms-win-crt-runtime-l1-1-0.dll
 0001:000058f4       ___vcrt_thread_attach      100068f4 f   MSVCRT:ucrt_stubs.obj
 0001:000058f4       ___scrt_stub_for_acrt_thread_attach 100068f4 f   MSVCRT:ucrt_stubs.obj
 0001:000058f4       ___scrt_stub_for_acrt_thread_detach 100068f4 f   MSVCRT:ucrt_stubs.obj
 0001:000058f4       ___scrt_stub_for_acrt_uninitialize 100068f4 f   MSVCRT:ucrt_stubs.obj
 0001:000058f4       ___scrt_stub_for_acrt_initialize 100068f4 f   MSVCRT:ucrt_stubs.obj
 0001:000058f4       ___vcrt_initialize         100068f4 f   MSVCRT:ucrt_stubs.obj
 0001:000058f4       ___scrt_stub_for_acrt_uninitialize_critical 100068f4 f   MSVCRT:ucrt_stubs.obj
 0001:000058f4       ___vcrt_uninitialize_critical 100068f4 f   MSVCRT:ucrt_stubs.obj
 0001:000058f4       ___vcrt_thread_detach      100068f4 f   MSVCRT:ucrt_stubs.obj
 0001:000058f4       ___acrt_uninitialize       100068f4 f   MSVCRT:ucrt_stubs.obj
 0001:000058f4       ___vcrt_uninitialize       100068f4 f   MSVCRT:ucrt_stubs.obj
 0001:000058f4       ___acrt_thread_detach      100068f4 f   MSVCRT:ucrt_stubs.obj
 0001:000058f4       ___acrt_uninitialize_critical 100068f4 f   MSVCRT:ucrt_stubs.obj
 0001:000058f4       ___acrt_initialize         100068f4 f   MSVCRT:ucrt_stubs.obj
 0001:000058f4       ___acrt_thread_attach      100068f4 f   MSVCRT:ucrt_stubs.obj
 0001:000058f7       ___scrt_stub_for_is_c_termination_complete 100068f7 f   MSVCRT:ucrt_stubs.obj
 0001:000058f7       __is_c_termination_complete 100068f7 f   MSVCRT:ucrt_stubs.obj
 0002:00000000       __imp__SetFileSecurityW@12 10007000     advapi32:ADVAPI32.dll
 0002:00000004       __imp__ConvertStringSidToSidW@8 10007004     advapi32:ADVAPI32.dll
 0002:00000008       __imp__ConvertSidToStringSidW@8 10007008     advapi32:ADVAPI32.dll
 0002:0000000c       __imp__LookupPrivilegeValueW@12 1000700c     advapi32:ADVAPI32.dll
 0002:00000010       __imp__LookupAccountNameW@28 10007010     advapi32:ADVAPI32.dll
 0002:00000014       __imp__LookupAccountSidW@28 10007014     advapi32:ADVAPI32.dll
 0002:00000018       __imp__SetSecurityDescriptorOwner@12 10007018     advapi32:ADVAPI32.dll
 0002:0000001c       __imp__SetSecurityDescriptorDacl@16 1000701c     advapi32:ADVAPI32.dll
 0002:00000020       __imp__MapGenericMask@8    10007020     advapi32:ADVAPI32.dll
 0002:00000024       __imp__InitializeSecurityDescriptor@8 10007024     advapi32:ADVAPI32.dll
 0002:00000028       __imp__InitializeAcl@12    10007028     advapi32:ADVAPI32.dll
 0002:0000002c       __imp__GetTokenInformation@20 1000702c     advapi32:ADVAPI32.dll
 0002:00000030       __imp__GetSecurityDescriptorOwner@12 10007030     advapi32:ADVAPI32.dll
 0002:00000034       __imp__GetSecurityDescriptorDacl@16 10007034     advapi32:ADVAPI32.dll
 0002:00000038       __imp__GetLengthSid@4      10007038     advapi32:ADVAPI32.dll
 0002:0000003c       __imp__GetFileSecurityW@20 1000703c     advapi32:ADVAPI32.dll
 0002:00000040       __imp__GetAclInformation@16 10007040     advapi32:ADVAPI32.dll
 0002:00000044       __imp__GetAce@12           10007044     advapi32:ADVAPI32.dll
 0002:00000048       __imp__DuplicateTokenEx@24 10007048     advapi32:ADVAPI32.dll
 0002:0000004c       __imp__AdjustTokenPrivileges@24 1000704c     advapi32:ADVAPI32.dll
 0002:00000050       __imp__AddAccessDeniedAceEx@20 10007050     advapi32:ADVAPI32.dll
 0002:00000054       __imp__AddAccessAllowedAceEx@20 10007054     advapi32:ADVAPI32.dll
 0002:00000058       __imp__AccessCheck@32      10007058     advapi32:ADVAPI32.dll
 0002:0000005c       __imp__OpenThreadToken@16  1000705c     advapi32:ADVAPI32.dll
 0002:00000060       __imp__OpenProcessToken@12 10007060     advapi32:ADVAPI32.dll
 0002:00000064       __imp__SetThreadToken@8    10007064     advapi32:ADVAPI32.dll
 0002:00000068       __imp__RegQueryValueExW@24 10007068     advapi32:ADVAPI32.dll
 0002:0000006c       __imp__RegOpenKeyExW@20    1000706c     advapi32:ADVAPI32.dll
 0002:00000070       __imp__RegCloseKey@4       10007070     advapi32:ADVAPI32.dll
 0002:00000074       \177ADVAPI32_NULL_THUNK_DATA 10007074     advapi32:ADVAPI32.dll
 0002:00000078       __imp__IsDebuggerPresent@0 10007078     kernel32:KERNEL32.dll
 0002:0000007c       __imp__InitializeSListHead@4 1000707c     kernel32:KERNEL32.dll
 0002:00000080       __imp__DisableThreadLibraryCalls@4 10007080     kernel32:KERNEL32.dll
 0002:00000084       __imp__GetSystemTimeAsFileTime@4 10007084     kernel32:KERNEL32.dll
 0002:00000088       __imp__GetCurrentThreadId@0 10007088     kernel32:KERNEL32.dll
 0002:0000008c       __imp__GetCurrentProcessId@0 1000708c     kernel32:KERNEL32.dll
 0002:00000090       __imp__IsProcessorFeaturePresent@4 10007090     kernel32:KERNEL32.dll
 0002:00000094       __imp__TerminateProcess@8  10007094     kernel32:KERNEL32.dll
 0002:00000098       __imp__SetUnhandledExceptionFilter@4 10007098     kernel32:KERNEL32.dll
 0002:0000009c       __imp__UnhandledExceptionFilter@4 1000709c     kernel32:KERNEL32.dll
 0002:000000a0       __imp__CreateSymbolicLinkW@12 100070a0     kernel32:KERNEL32.dll
 0002:000000a4       __imp__ReadDirectoryChangesW@32 100070a4     kernel32:KERNEL32.dll
 0002:000000a8       __imp__CreateHardLinkW@12  100070a8     kernel32:KERNEL32.dll
 0002:000000ac       __imp__CreateDirectoryW@8  100070ac     kernel32:KERNEL32.dll
 0002:000000b0       __imp__CreateFileW@28      100070b0     kernel32:KERNEL32.dll
 0002:000000b4       __imp__DeleteFileW@4       100070b4     kernel32:KERNEL32.dll
 0002:000000b8       __imp__FindClose@4         100070b8     kernel32:KERNEL32.dll
 0002:000000bc       __imp__FindFirstFileW@8    100070bc     kernel32:KERNEL32.dll
 0002:000000c0       __imp__FindNextFileW@8     100070c0     kernel32:KERNEL32.dll
 0002:000000c4       __imp__GetDiskFreeSpaceExW@16 100070c4     kernel32:KERNEL32.dll
 0002:000000c8       __imp__GetDriveTypeW@4     100070c8     kernel32:KERNEL32.dll
 0002:000000cc       __imp__GetFileAttributesW@4 100070cc     kernel32:KERNEL32.dll
 0002:000000d0       __imp__GetFileAttributesExW@12 100070d0     kernel32:KERNEL32.dll
 0002:000000d4       __imp__GetFinalPathNameByHandleW@16 100070d4     kernel32:KERNEL32.dll
 0002:000000d8       __imp__GetFullPathNameW@16 100070d8     kernel32:KERNEL32.dll
 0002:000000dc       __imp__GetLogicalDrives@0  100070dc     kernel32:KERNEL32.dll
 0002:000000e0       __imp__GetVolumeInformationW@32 100070e0     kernel32:KERNEL32.dll
 0002:000000e4       __imp__GetVolumePathNameW@12 100070e4     kernel32:KERNEL32.dll
 0002:000000e8       __imp__RemoveDirectoryW@4  100070e8     kernel32:KERNEL32.dll
 0002:000000ec       __imp__SetEndOfFile@4      100070ec     kernel32:KERNEL32.dll
 0002:000000f0       __imp__SetFileAttributesW@8 100070f0     kernel32:KERNEL32.dll
 0002:000000f4       __imp__SetFileTime@16      100070f4     kernel32:KERNEL32.dll
 0002:000000f8       __imp__FindFirstStreamW@16 100070f8     kernel32:KERNEL32.dll
 0002:000000fc       __imp__FindNextStreamW@8   100070fc     kernel32:KERNEL32.dll
 0002:00000100       __imp__LockFileEx@24       10007100     kernel32:KERNEL32.dll
 0002:00000104       __imp__DeviceIoControl@32  10007104     kernel32:KERNEL32.dll
 0002:00000108       __imp__CancelIo@4          10007108     kernel32:KERNEL32.dll
 0002:0000010c       __imp__CreateEventW@16     1000710c     kernel32:KERNEL32.dll
 0002:00000110       __imp__GetCurrentThread@0  10007110     kernel32:KERNEL32.dll
 0002:00000114       __imp__LocalAlloc@8        10007114     kernel32:KERNEL32.dll
 0002:00000118       __imp__LocalFree@4         10007118     kernel32:KERNEL32.dll
 0002:0000011c       __imp__CopyFileExW@24      1000711c     kernel32:KERNEL32.dll
 0002:00000120       __imp__QueryPerformanceCounter@4 10007120     kernel32:KERNEL32.dll
 0002:00000124       __imp__SetHandleInformation@12 10007124     kernel32:KERNEL32.dll
 0002:00000128       __imp__FlushViewOfFile@8   10007128     kernel32:KERNEL32.dll
 0002:0000012c       __imp__SetFilePointerEx@20 1000712c     kernel32:KERNEL32.dll
 0002:00000130       __imp__CloseHandle@4       10007130     kernel32:KERNEL32.dll
 0002:00000134       __imp__GetLastError@0      10007134     kernel32:KERNEL32.dll
 0002:00000138       __imp__GetSystemInfo@4     10007138     kernel32:KERNEL32.dll
 0002:0000013c       __imp__MapViewOfFile@20    1000713c     kernel32:KERNEL32.dll
 0002:00000140       __imp__UnmapViewOfFile@4   10007140     kernel32:KERNEL32.dll
 0002:00000144       __imp__CreateFileMappingA@24 10007144     kernel32:KERNEL32.dll
 0002:00000148       __imp__FlushFileBuffers@4  10007148     kernel32:KERNEL32.dll
 0002:0000014c       __imp__GetDiskFreeSpaceW@20 1000714c     kernel32:KERNEL32.dll
 0002:00000150       __imp__GetFileSizeEx@8     10007150     kernel32:KERNEL32.dll
 0002:00000154       __imp__FormatMessageW@28   10007154     kernel32:KERNEL32.dll
 0002:00000158       __imp__ReadFile@20         10007158     kernel32:KERNEL32.dll
 0002:0000015c       __imp__SetFileInformationByHandle@16 1000715c     kernel32:KERNEL32.dll
 0002:00000160       __imp__UnlockFileEx@20     10007160     kernel32:KERNEL32.dll
 0002:00000164       __imp__WriteFile@20        10007164     kernel32:KERNEL32.dll
 0002:00000168       __imp__DuplicateHandle@28  10007168     kernel32:KERNEL32.dll
 0002:0000016c       __imp__GetOverlappedResult@16 1000716c     kernel32:KERNEL32.dll
 0002:00000170       __imp__GetCurrentProcess@0 10007170     kernel32:KERNEL32.dll
 0002:00000174       __imp__ReOpenFile@16       10007174     kernel32:KERNEL32.dll
 0002:00000178       __imp__GetFileInformationByHandle@8 10007178     kernel32:KERNEL32.dll
 0002:0000017c       __imp__CreateIoCompletionPort@16 1000717c     kernel32:KERNEL32.dll
 0002:00000180       __imp__GetQueuedCompletionStatus@20 10007180     kernel32:KERNEL32.dll
 0002:00000184       __imp__PostQueuedCompletionStatus@16 10007184     kernel32:KERNEL32.dll
 0002:00000188       __imp__MoveFileExW@12      10007188     kernel32:KERNEL32.dll
 0002:0000018c       \177KERNEL32_NULL_THUNK_DATA 1000718c     kernel32:KERNEL32.dll
 0002:00000190       __imp__TransmitFile@28     10007190     Mswsock:MSWSOCK.dll
 0002:00000194       \177MSWSOCK_NULL_THUNK_DATA 10007194     Mswsock:MSWSOCK.dll
 0002:00000198       __imp____std_type_info_destroy_list 10007198     vcruntime:VCRUNTIME140.dll
 0002:0000019c       __imp___except_handler4_common 1000719c     vcruntime:VCRUNTIME140.dll
 0002:000001a0       __imp__memset              100071a0     vcruntime:VCRUNTIME140.dll
 0002:000001a4       \177VCRUNTIME140_NULL_THUNK_DATA 100071a4     vcruntime:VCRUNTIME140.dll
 0002:000001a8       __imp__recv@16             100071a8     ws2_32:WS2_32.dll
 0002:000001ac       __imp__closesocket@4       100071ac     ws2_32:WS2_32.dll
 0002:000001b0       __imp__send@16             100071b0     ws2_32:WS2_32.dll
 0002:000001b4       __imp__accept@12           100071b4     ws2_32:WS2_32.dll
 0002:000001b8       __imp__socket@12           100071b8     ws2_32:WS2_32.dll
 0002:000001bc       __imp__shutdown@8          100071bc     ws2_32:WS2_32.dll
 0002:000001c0       __imp__setsockopt@20       100071c0     ws2_32:WS2_32.dll
 0002:000001c4       __imp__ntohl@4             100071c4     ws2_32:WS2_32.dll
 0002:000001c8       __imp__listen@8            100071c8     ws2_32:WS2_32.dll
 0002:000001cc       __imp__htonl@4             100071cc     ws2_32:WS2_32.dll
 0002:000001d0       __imp__getsockopt@20       100071d0     ws2_32:WS2_32.dll
 0002:000001d4       __imp__getsockname@12      100071d4     ws2_32:WS2_32.dll
 0002:000001d8       __imp__getpeername@12      100071d8     ws2_32:WS2_32.dll
 0002:000001dc       __imp____WSAFDIsSet@8      100071dc     ws2_32:WS2_32.dll
 0002:000001e0       __imp__WSAEventSelect@12   100071e0     ws2_32:WS2_32.dll
 0002:000001e4       __imp__ioctlsocket@12      100071e4     ws2_32:WS2_32.dll
 0002:000001e8       __imp__WSASend@28          100071e8     ws2_32:WS2_32.dll
 0002:000001ec       __imp__WSARecv@28          100071ec     ws2_32:WS2_32.dll
 0002:000001f0       __imp__WSAIoctl@36         100071f0     ws2_32:WS2_32.dll
 0002:000001f4       __imp__WSAGetLastError@0   100071f4     ws2_32:WS2_32.dll
 0002:000001f8       __imp__sendto@24           100071f8     ws2_32:WS2_32.dll
 0002:000001fc       __imp__select@20           100071fc     ws2_32:WS2_32.dll
 0002:00000200       __imp__recvfrom@24         10007200     ws2_32:WS2_32.dll
 0002:00000204       __imp__connect@12          10007204     ws2_32:WS2_32.dll
 0002:00000208       \177WS2_32_NULL_THUNK_DATA 10007208     ws2_32:WS2_32.dll
 0002:0000020c       __imp__malloc              1000720c     ucrt:api-ms-win-crt-heap-l1-1-0.dll
 0002:00000210       __imp__free                10007210     ucrt:api-ms-win-crt-heap-l1-1-0.dll
 0002:00000214       \177api-ms-win-crt-heap-l1-1-0_NULL_THUNK_DATA 10007214     ucrt:api-ms-win-crt-heap-l1-1-0.dll
 0002:00000218       __imp___execute_onexit_table 10007218     ucrt:api-ms-win-crt-runtime-l1-1-0.dll
 0002:0000021c       __imp___initialize_onexit_table 1000721c     ucrt:api-ms-win-crt-runtime-l1-1-0.dll
 0002:00000220       __imp___configure_narrow_argv 10007220     ucrt:api-ms-win-crt-runtime-l1-1-0.dll
 0002:00000224       __imp___seh_filter_dll     10007224     ucrt:api-ms-win-crt-runtime-l1-1-0.dll
 0002:00000228       __imp___initterm_e         10007228     ucrt:api-ms-win-crt-runtime-l1-1-0.dll
 0002:0000022c       __imp___initterm           1000722c     ucrt:api-ms-win-crt-runtime-l1-1-0.dll
 0002:00000230       __imp___errno              10007230     ucrt:api-ms-win-crt-runtime-l1-1-0.dll
 0002:00000234       __imp___cexit              10007234     ucrt:api-ms-win-crt-runtime-l1-1-0.dll
 0002:00000238       __imp___initialize_narrow_environment 10007238     ucrt:api-ms-win-crt-runtime-l1-1-0.dll
 0002:0000023c       \177api-ms-win-crt-runtime-l1-1-0_NULL_THUNK_DATA 1000723c     ucrt:api-ms-win-crt-runtime-l1-1-0.dll
 0002:00000240       __imp___get_osfhandle      10007240     ucrt:api-ms-win-crt-stdio-l1-1-0.dll
 0002:00000244       \177api-ms-win-crt-stdio-l1-1-0_NULL_THUNK_DATA 10007244     ucrt:api-ms-win-crt-stdio-l1-1-0.dll
 0002:00000248       __imp__wcslen              10007248     ucrt:api-ms-win-crt-string-l1-1-0.dll
 0002:0000024c       \177api-ms-win-crt-string-l1-1-0_NULL_THUNK_DATA 1000724c     ucrt:api-ms-win-crt-string-l1-1-0.dll
 0002:00000250       __imp__JNU_ThrowIOExceptionWithLastError@8 10007250     java:java.dll
 0002:00000254       __imp__JNU_ThrowByName@12  10007254     java:java.dll
 0002:00000258       __imp__JNU_NewObjectByName 10007258     java:java.dll
 0002:0000025c       __imp__JNU_ThrowInternalError@8 1000725c     java:java.dll
 0002:00000260       __imp__Java_sun_security_provider_NativeSeedGenerator_nativeGenerateSeed@12 10007260     java:java.dll
 0002:00000264       __imp__JNU_ThrowOutOfMemoryError@8 10007264     java:java.dll
 0002:00000268       \177java_NULL_THUNK_DATA   10007268     java:java.dll
 0002:0000026c       __imp__NET_InetAddressToSockaddr@24 1000726c     net:net.dll
 0002:00000270       __imp__NET_SockaddrEqualsInetAddress@12 10007270     net:net.dll
 0002:00000274       __imp__NET_WinBind@16      10007274     net:net.dll
 0002:00000278       __imp__NET_EnableFastTcpLoopbackConnect@4 10007278     net:net.dll
 0002:0000027c       __imp__initInetAddressIDs@4 1000727c     net:net.dll
 0002:00000280       __imp__NET_ThrowNew@12     10007280     net:net.dll
 0002:00000284       __imp__ipv6_available@0    10007284     net:net.dll
 0002:00000288       __imp__NET_GetSockOpt@20   10007288     net:net.dll
 0002:0000028c       __imp__NET_SetSockOpt@20   1000728c     net:net.dll
 0002:00000290       __imp__NET_EnableFastTcpLoopback@4 10007290     net:net.dll
 0002:00000294       __imp__NET_SockaddrToInetAddress@12 10007294     net:net.dll
 0002:00000298       __imp__NET_GetPortFromSockaddr@4 10007298     net:net.dll
 0002:0000029c       \177net_NULL_THUNK_DATA    1000729c     net:net.dll
 0002:000002a0       ___guard_check_icall_fptr  100072a0     MSVCRT:guard_support.obj
 0002:000002a4       ___xc_a                    100072a4     MSVCRT:initializers.obj
 0002:000002a8       ___xc_z                    100072a8     MSVCRT:initializers.obj
 0002:000002ac       ___xi_a                    100072ac     MSVCRT:initializers.obj
 0002:000002b0       ___xi_z                    100072b0     MSVCRT:initializers.obj
 0002:000002b4       ___xp_a                    100072b4     MSVCRT:initializers.obj
 0002:000002b8       ___xp_z                    100072b8     MSVCRT:initializers.obj
 0002:000002bc       ___xt_a                    100072bc     MSVCRT:initializers.obj
 0002:000002c0       ___xt_z                    100072c0     MSVCRT:initializers.obj
 0002:000002d0       ??_C@_0BL@HBNNAPLM@java?1net?1InetSocketAddress@ 100072d0     DatagramChannelImpl.obj
 0002:000002ec       ??_C@_0BL@KCCEIBDI@?$CILjava?1net?1InetAddress?$DLI?$CJV@ 100072ec     DatagramChannelImpl.obj
 0002:00000308       ??_C@_06FALKBLGB@?$DMinit?$DO@ 10007308     DatagramChannelImpl.obj
 0002:00000310       ??_C@_0BP@BNFFMBJL@sun?1nio?1ch?1DatagramChannelImpl@ 10007310     DatagramChannelImpl.obj
 0002:00000330       ??_C@_0BJ@NDFGGFKE@Ljava?1net?1SocketAddress?$DL@ 10007330     DatagramChannelImpl.obj
 0002:0000034c       ??_C@_06CGHJMPBJ@sender@   1000734c     DatagramChannelImpl.obj
 0002:00000354       ??_C@_0BH@FIKCFBLO@Ljava?1net?1InetAddress?$DL@ 10007354     DatagramChannelImpl.obj
 0002:0000036c       ??_C@_0BI@OANHFGOF@cachedSenderInetAddress@ 1000736c     DatagramChannelImpl.obj
 0002:00000384       ??_C@_01JPJNBJEM@I@        10007384     DatagramChannelImpl.obj
 0002:00000388       ??_C@_0BB@JLIPPJNN@cachedSenderPort@ 10007388     DatagramChannelImpl.obj
 0002:0000039c       ??_C@_0CC@BDDMPFBF@java?1net?1PortUnreachableExcepti@ 1000739c     DatagramChannelImpl.obj
 0002:000003c0       ??_C@_0P@DGIIHHAE@WSARecv?5failed@ 100073c0     DatagramDispatcher.obj
 0002:000003d0       ??_C@_0P@NKOFNKCM@WSASend?5failed@ 100073d0     DatagramDispatcher.obj
 0002:000003e0       ??_C@_0BJ@BDFOFHPL@Ljava?1io?1FileDescriptor?$DL@ 100073e0     FileChannelImpl.obj
 0002:000003fc       ??_C@_02ENHFDPNM@fd@       100073fc     FileChannelImpl.obj
 0002:00000400       ??_C@_0L@DPMFILPJ@Map?5failed@ 10007400     FileChannelImpl.obj
 0002:0000040c       ??_C@_0N@IGMMIDE@Unmap?5failed@ 1000740c     FileChannelImpl.obj
 0002:0000041c       ??_C@_0BI@ICELLBHO@SetFilePointerEx?5failed@ 1000741c     FileChannelImpl.obj
 0002:00000434       ??_C@_0BA@CJMHIODJ@transfer?5failed@ 10007434     FileChannelImpl.obj
 0002:00000444       ??_C@_0P@EFDAIKIF@Invalid?5handle@ 10007444     FileDispatcherImpl.obj
 0002:00000454       ??_C@_0M@DCKEEFAG@Read?5failed@ 10007454     FileDispatcherImpl.obj
 0002:00000460       ??_C@_0M@HPFDGGMC@Seek?5failed@ 10007460     FileDispatcherImpl.obj
 0002:0000046c       ??_C@_0N@PGCLODBC@Write?5failed@ 1000746c     FileDispatcherImpl.obj
 0002:0000047c       ??_C@_0N@EFKIKJEB@Force?5failed@ 1000747c     FileDispatcherImpl.obj
 0002:0000048c       ??_C@_0BC@FODOCFKM@Truncation?5failed@ 1000748c     FileDispatcherImpl.obj
 0002:000004a0       ??_C@_0M@GLCOPFPC@Size?5failed@ 100074a0     FileDispatcherImpl.obj
 0002:000004ac       ??_C@_0M@OOGODMIM@Lock?5failed@ 100074ac     FileDispatcherImpl.obj
 0002:000004b8       ??_C@_0P@MAMCLOFD@Release?5failed@ 100074b8     FileDispatcherImpl.obj
 0002:000004c8       ??_C@_0N@GNNFMAIG@Close?5failed@ 100074c8     FileDispatcherImpl.obj
 0002:000004d8       ??_C@_0BH@OPJFPPPK@DuplicateHandle?5failed@ 100074d8     FileDispatcherImpl.obj
 0002:000004f0       ??_C@_0BG@JDMBHIAK@DirectIO?5setup?5failed@ 100074f0     FileDispatcherImpl.obj
 0002:00000508       ??_C@_01LELAEKIP@J@        10007508     FileKey.obj
 0002:0000050c       ??_C@_0BF@GJBBDEBO@dwVolumeSerialNumber@ 1000750c     FileKey.obj
 0002:00000524       ??_C@_0P@OJOGHFHE@nFileIndexHigh@ 10007524     FileKey.obj
 0002:00000534       ??_C@_0O@HJEFBNI@nFileIndexLow@ 10007534     FileKey.obj
 0002:00000544       ??_C@_0CC@EJDNCKME@GetFileInformationByHandle?5fail@ 10007544     FileKey.obj
 0002:00000568       ??_C@_0BH@MPHCPCAM@java?1io?1FileDescriptor@ 10007568     IOUtil.obj
 0002:00000580       ??_C@_06NCGDPKCC@handle@   10007580     IOUtil.obj
 0002:00000588       ??_C@_0BC@PPBACNOJ@Read?1write?5failed@ 10007588     IOUtil.obj
 0002:0000059c       ??_C@_05GGAEIDGJ@Drain@    1000759c     IOUtil.obj
 0002:000005a4       ??_C@_0CB@EANIAHBH@sun?1nio?1ch?1Iocp$CompletionStatu@ 100075a4     Iocp.obj
 0002:000005c8       ??_C@_05KKCIMGE@error@     100075c8     Iocp.obj
 0002:000005d0       ??_C@_0BB@LMCKIICB@bytesTransferred@ 100075d0     Iocp.obj
 0002:000005e4       ??_C@_0O@HHOLMKBG@completionKey@ 100075e4     Iocp.obj
 0002:000005f4       ??_C@_0L@GFMJGGB@overlapped@ 100075f4     Iocp.obj
 0002:00000600       ??_C@_0BO@HNKCMKLP@CreateIoCompletionPort?5failed@ 10007600     Iocp.obj
 0002:00000620       ??_C@_0CB@GOEOMHMA@GetQueuedCompletionStatus?5faile@ 10007620     Iocp.obj
 0002:00000644       ??_C@_0BL@IDOBBHMP@PostQueuedCompletionStatus@ 10007644     Iocp.obj
 0002:00000660       ??_C@_0N@MNOMAIIN@Flush?5failed@ 10007660     MappedByteBuffer.obj
 0002:00000670       ??_C@_06HBELJPBO@socket@   10007670     Net.obj
 0002:00000678       ??_C@_0N@JOEJINBO@fastLoopback@ 10007678     Net.obj
 0002:00000688       ??_C@_04NPNJNMMP@bind@     10007688     Net.obj
 0002:00000690       ??_C@_06OODDLKLE@listen@   10007690     Net.obj
 0002:00000698       ??_C@_07KAIBNCHO@connect@  10007698     Net.obj
 0002:000006a0       ??_C@_0M@ODFENJLC@getsockname@ 100076a0     Net.obj
 0002:000006ac       ??_C@_08FIACBBDA@shutdown@ 100076ac     Net.obj
 0002:000006b8       ??_C@_0O@BMGFIIHF@Accept?5failed@ 100076b8     ServerSocketChannelImpl.obj
 0002:000006c8       ??_C@_0BF@LNJHKELF@java?1net?1InetAddress@ 100076c8     SocketChannelImpl.obj
 0002:000006e0       ??_C@_07LHEPONKL@address@  100076e0     SocketChannelImpl.obj
 0002:000006e8       ??_C@_0L@DEFCDCGF@getsockopt@ 100076e8     SocketChannelImpl.obj
 0002:000006f4       ??_C@_0BD@MOAOKNAP@Vector?5read?5failed@ 100076f4     SocketDispatcher.obj
 0002:00000708       ??_C@_0BE@IPALPBFO@Vector?5write?5failed@ 10007708     SocketDispatcher.obj
 0002:0000071c       ??_C@_0BE@EFPANNNH@Socket?5close?5failed@ 1000771c     SocketDispatcher.obj
 0002:00000730       ??_C@_0BA@KDJDNLHD@ReadFile?5failed@ 10007730     WindowsAsynchronousFileChannelImpl.obj
 0002:00000740       ??_C@_0BB@IBAPLIEE@WriteFile?5failed@ 10007740     WindowsAsynchronousFileChannelImpl.obj
 0002:00000754       ??_C@_0O@FPJGNADN@socket?5failed@ 10007754     WindowsAsynchronousServerSocketChannelImpl.obj
 0002:00000764       ??_C@_0BA@PBEMOOLP@WSAIoctl?5failed@ 10007764     WindowsAsynchronousServerSocketChannelImpl.obj
 0002:00000774       ??_C@_0BA@CMPAPNB@AcceptEx?5failed@ 10007774     WindowsAsynchronousServerSocketChannelImpl.obj
 0002:00000784       ??_C@_0BD@FFLNFFAC@closesocket?5failed@ 10007784     WindowsAsynchronousServerSocketChannelImpl.obj
 0002:00000798       ??_C@_0BB@COIIDLME@ConnectEx?5failed@ 10007798     WindowsAsynchronousSocketChannelImpl.obj
 0002:000007ac       ??_C@_0BA@GMHHDNNI@shutdown?5failed@ 100077ac     WindowsAsynchronousSocketChannelImpl.obj
 0002:000007bc       ??_C@_04PFANPMCN@?$CII?$CJV@ 100077bc     WindowsNativeDispatcher.obj
 0002:000007c4       ??_C@_0BM@FOMEEEOI@sun?1nio?1fs?1WindowsException@ 100077c4     WindowsNativeDispatcher.obj
 0002:000007e0       ??_C@_0CN@IAHHKCCP@sun?1nio?1fs?1WindowsNativeDispatc@ 100077e0     WindowsNativeDispatcher.obj
 0002:00000810       ??_C@_0BD@JFADHEFE@Ljava?1lang?1String?$DL@ 10007810     WindowsNativeDispatcher.obj
 0002:00000824       ??_C@_04MEMAJGDJ@name@     10007824     WindowsNativeDispatcher.obj
 0002:0000082c       ??_C@_0L@HNMJPKNA@attributes@ 1000782c     WindowsNativeDispatcher.obj
 0002:00000838       ??_C@_0CP@OGPMEFOM@sun?1nio?1fs?1WindowsNativeDispatc@ 10007838     WindowsNativeDispatcher.obj
 0002:00000868       ??_C@_0DF@OBLOOIFM@sun?1nio?1fs?1WindowsNativeDispatc@ 10007868     WindowsNativeDispatcher.obj
 0002:000008a0       ??_C@_0P@BFNHNOMJ@fileSystemName@ 100078a0     WindowsNativeDispatcher.obj
 0002:000008b0       ??_C@_0L@HCGAGGAJ@volumeName@ 100078b0     WindowsNativeDispatcher.obj
 0002:000008bc       ??_C@_0BD@ILMPNPNH@volumeSerialNumber@ 100078bc     WindowsNativeDispatcher.obj
 0002:000008d0       ??_C@_05GECEPKB@flags@     100078d0     WindowsNativeDispatcher.obj
 0002:000008d8       ??_C@_0DB@OGAJBKPO@sun?1nio?1fs?1WindowsNativeDispatc@ 100078d8     WindowsNativeDispatcher.obj
 0002:0000090c       ??_C@_0BD@LDNCHAFG@freeBytesAvailable@ 1000790c     WindowsNativeDispatcher.obj
 0002:00000920       ??_C@_0BD@FIEGHADN@totalNumberOfBytes@ 10007920     WindowsNativeDispatcher.obj
 0002:00000934       ??_C@_0BH@DLDLDEPI@totalNumberOfFreeBytes@ 10007934     WindowsNativeDispatcher.obj
 0002:0000094c       ??_C@_0P@EEANGJCF@bytesPerSector@ 1000794c     WindowsNativeDispatcher.obj
 0002:0000095c       ??_C@_0CL@IEKIAJIE@sun?1nio?1fs?1WindowsNativeDispatc@ 1000795c     WindowsNativeDispatcher.obj
 0002:00000988       ??_C@_06LKIIGAOE@domain@   10007988     WindowsNativeDispatcher.obj
 0002:00000990       ??_C@_03MMGHDJKG@use@      10007990     WindowsNativeDispatcher.obj
 0002:00000994       ??_C@_0DC@CMOGENGN@sun?1nio?1fs?1WindowsNativeDispatc@ 10007994     WindowsNativeDispatcher.obj
 0002:000009c8       ??_C@_08BCFBCIIE@aceCount@ 100079c8     WindowsNativeDispatcher.obj
 0002:000009d4       ??_C@_0DE@MGDINMHA@sun?1nio?1fs?1WindowsNativeDispatc@ 100079d4     WindowsNativeDispatcher.obj
 0002:00000a08       ??_C@_0CC@NMODGIKH@Unable?5to?5allocate?5LUID?5structu@ 10007a08     WindowsNativeDispatcher.obj
 0002:00000a2c       ??_C@_0BI@COMCEALI@GetFullPathNameW?5failed@ 10007a2c     WindowsNativeDispatcher.obj
 0002:00000a44       ??_C@_0CB@DJOGFDBC@native?5memory?5allocation?5failur@ 10007a44     WindowsNativeDispatcher.obj
 0002:00000a68       ??_C@_0CB@BLMDNHEM@GetFinalPathNameByHandleW?5faile@ 10007a68     WindowsNativeDispatcher.obj
 0002:00000a8c       __pRawDllMain              10007a8c     MSVCRT:dll_dllmain.obj
 0002:00000a8c       __pDefaultRawDllMain       10007a8c     MSVCRT:dll_dllmain.obj
 0002:00000b10       __load_config_used         10007b10     MSVCRT:loadcfg.obj
 0002:00000bb0       ___safe_se_handler_table   10007bb0     <linker-defined>
 0002:00000e34       ___rtc_iaa                 10007e34     MSVCRT:initsect.obj
 0002:00000e38       ___rtc_izz                 10007e38     MSVCRT:initsect.obj
 0002:00000e3c       ___rtc_taa                 10007e3c     MSVCRT:initsect.obj
 0002:00000e40       ___rtc_tzz                 10007e40     MSVCRT:initsect.obj
 0002:000039f8       __IMPORT_DESCRIPTOR_WS2_32 1000a9f8     ws2_32:WS2_32.dll
 0002:00003a0c       __IMPORT_DESCRIPTOR_java   1000aa0c     java:java.dll
 0002:00003a20       __IMPORT_DESCRIPTOR_net    1000aa20     net:net.dll
 0002:00003a34       __IMPORT_DESCRIPTOR_ADVAPI32 1000aa34     advapi32:ADVAPI32.dll
 0002:00003a48       __IMPORT_DESCRIPTOR_MSWSOCK 1000aa48     Mswsock:MSWSOCK.dll
 0002:00003a5c       __IMPORT_DESCRIPTOR_KERNEL32 1000aa5c     kernel32:KERNEL32.dll
 0002:00003a70       __IMPORT_DESCRIPTOR_VCRUNTIME140 1000aa70     vcruntime:VCRUNTIME140.dll
 0002:00003a84       __IMPORT_DESCRIPTOR_api-ms-win-crt-heap-l1-1-0 1000aa84     ucrt:api-ms-win-crt-heap-l1-1-0.dll
 0002:00003a98       __IMPORT_DESCRIPTOR_api-ms-win-crt-stdio-l1-1-0 1000aa98     ucrt:api-ms-win-crt-stdio-l1-1-0.dll
 0002:00003aac       __IMPORT_DESCRIPTOR_api-ms-win-crt-string-l1-1-0 1000aaac     ucrt:api-ms-win-crt-string-l1-1-0.dll
 0002:00003ac0       __IMPORT_DESCRIPTOR_api-ms-win-crt-runtime-l1-1-0 1000aac0     ucrt:api-ms-win-crt-runtime-l1-1-0.dll
 0002:00003ad4       __NULL_IMPORT_DESCRIPTOR   1000aad4     ws2_32:WS2_32.dll
 0003:00000004       ___security_cookie_complement 1000c004     MSVCRT:gs_cookie.obj
 0003:00000008       ___security_cookie         1000c008     MSVCRT:gs_cookie.obj
 0003:00000010       ___scrt_native_dllmain_reason 1000c010     MSVCRT:utility.obj
 0003:00000020       ___isa_enabled             1000c020     MSVCRT:cpu_disp.obj
 0003:00000024       ___scrt_ucrt_dll_is_in_use 1000c024     MSVCRT:ucrt_stubs.obj
 0003:00000400       ?__type_info_root_node@@3U__type_info_node@@A 1000c400     MSVCRT:tncleanup.obj
 0003:00000408       ?_OptionsStorage@?1??__local_stdio_printf_options@@9@4_KA 1000c408     MSVCRT:default_local_stdio_options.obj
 0003:00000410       ?_OptionsStorage@?1??__local_stdio_scanf_options@@9@4_KA 1000c410     MSVCRT:default_local_stdio_options.obj
 0003:00000418       ___scrt_current_native_startup_state 1000c418     MSVCRT:utility.obj
 0003:0000041c       ___scrt_native_startup_lock 1000c41c     MSVCRT:utility.obj
 0003:0000043c       ___scrt_debugger_hook_flag 1000c43c     MSVCRT:utility_desktop.obj
 0003:00000440       ___isa_available           1000c440     MSVCRT:cpu_disp.obj
 0003:00000444       ___favor                   1000c444     MSVCRT:cpu_disp.obj
 0003:00000448       ___dyn_tls_init_callback   1000c448     <common>

 entry point at        0001:00004fc2

 Static symbols

 0000:ffff1000       .debug$S                   10000000     kernel32:KERNEL32.dll
 0000:ffff1000       .debug$S                   10000000     ws2_32:WS2_32.dll
 0000:ffff1000       .debug$S                   10000000     ws2_32:WS2_32.dll
 0000:ffff1000       .debug$S                   10000000     ws2_32:WS2_32.dll
 0000:ffff1000       .debug$S                   10000000     ws2_32:WS2_32.dll
 0000:ffff1000       .debug$S                   10000000     ws2_32:WS2_32.dll
 0000:ffff1000       .debug$S                   10000000     ws2_32:WS2_32.dll
 0000:ffff1000       .debug$S                   10000000     ws2_32:WS2_32.dll
 0000:ffff1000       .debug$S                   10000000     ws2_32:WS2_32.dll
 0000:ffff1000       .debug$S                   10000000     ws2_32:WS2_32.dll
 0000:ffff1000       .debug$S                   10000000     ws2_32:WS2_32.dll
 0000:ffff1000       .debug$S                   10000000     ws2_32:WS2_32.dll
 0000:ffff1000       .debug$S                   10000000     ws2_32:WS2_32.dll
 0000:ffff1000       .debug$S                   10000000     ws2_32:WS2_32.dll
 0000:ffff1000       .debug$S                   10000000     ws2_32:WS2_32.dll
 0000:ffff1000       .debug$S                   10000000     ws2_32:WS2_32.dll
 0000:ffff1000       .debug$S                   10000000     ws2_32:WS2_32.dll
 0000:ffff1000       .debug$S                   10000000     ws2_32:WS2_32.dll
 0000:ffff1000       .debug$S                   10000000     ws2_32:WS2_32.dll
 0000:ffff1000       .debug$S                   10000000     ws2_32:WS2_32.dll
 0000:ffff1000       .debug$S                   10000000     ws2_32:WS2_32.dll
 0000:ffff1000       .debug$S                   10000000     java:java.dll
 0000:ffff1000       .debug$S                   10000000     java:java.dll
 0000:ffff1000       .debug$S                   10000000     java:java.dll
 0000:ffff1000       .debug$S                   10000000     java:java.dll
 0000:ffff1000       .debug$S                   10000000     java:java.dll
 0000:ffff1000       .debug$S                   10000000     java:java.dll
 0000:ffff1000       .debug$S                   10000000     net:net.dll
 0000:ffff1000       .debug$S                   10000000     net:net.dll
 0000:ffff1000       .debug$S                   10000000     net:net.dll
 0000:ffff1000       .debug$S                   10000000     net:net.dll
 0000:ffff1000       .debug$S                   10000000     net:net.dll
 0000:ffff1000       .debug$S                   10000000     net:net.dll
 0000:ffff1000       .debug$S                   10000000     net:net.dll
 0000:ffff1000       .debug$S                   10000000     net:net.dll
 0000:ffff1000       .debug$S                   10000000     net:net.dll
 0000:ffff1000       .debug$S                   10000000     net:net.dll
 0000:ffff1000       .debug$S                   10000000     net:net.dll
 0000:ffff1000       .debug$S                   10000000     net:net.dll
 0000:ffff1000       .debug$S                   10000000     advapi32:ADVAPI32.dll
 0000:ffff1000       .debug$S                   10000000     advapi32:ADVAPI32.dll
 0000:ffff1000       .debug$S                   10000000     advapi32:ADVAPI32.dll
 0000:ffff1000       .debug$S                   10000000     advapi32:ADVAPI32.dll
 0000:ffff1000       .debug$S                   10000000     advapi32:ADVAPI32.dll
 0000:ffff1000       .debug$S                   10000000     advapi32:ADVAPI32.dll
 0000:ffff1000       .debug$S                   10000000     advapi32:ADVAPI32.dll
 0000:ffff1000       .debug$S                   10000000     advapi32:ADVAPI32.dll
 0000:ffff1000       .debug$S                   10000000     advapi32:ADVAPI32.dll
 0000:ffff1000       .debug$S                   10000000     advapi32:ADVAPI32.dll
 0000:ffff1000       .debug$S                   10000000     advapi32:ADVAPI32.dll
 0000:ffff1000       .debug$S                   10000000     advapi32:ADVAPI32.dll
 0000:ffff1000       .debug$S                   10000000     advapi32:ADVAPI32.dll
 0000:ffff1000       .debug$S                   10000000     advapi32:ADVAPI32.dll
 0000:ffff1000       .debug$S                   10000000     advapi32:ADVAPI32.dll
 0000:ffff1000       .debug$S                   10000000     advapi32:ADVAPI32.dll
 0000:ffff1000       .debug$S                   10000000     advapi32:ADVAPI32.dll
 0000:ffff1000       .debug$S                   10000000     advapi32:ADVAPI32.dll
 0000:ffff1000       .debug$S                   10000000     advapi32:ADVAPI32.dll
 0000:ffff1000       .debug$S                   10000000     advapi32:ADVAPI32.dll
 0000:ffff1000       .debug$S                   10000000     advapi32:ADVAPI32.dll
 0000:ffff1000       .debug$S                   10000000     advapi32:ADVAPI32.dll
 0000:ffff1000       .debug$S                   10000000     advapi32:ADVAPI32.dll
 0000:ffff1000       .debug$S                   10000000     advapi32:ADVAPI32.dll
 0000:ffff1000       .debug$S                   10000000     advapi32:ADVAPI32.dll
 0000:ffff1000       .debug$S                   10000000     advapi32:ADVAPI32.dll
 0000:ffff1000       .debug$S                   10000000     advapi32:ADVAPI32.dll
 0000:ffff1000       .debug$S                   10000000     advapi32:ADVAPI32.dll
 0000:ffff1000       .debug$S                   10000000     advapi32:ADVAPI32.dll
 0000:ffff1000       .debug$S                   10000000     ws2_32:WS2_32.dll
 0000:ffff1000       .debug$S                   10000000     ws2_32:WS2_32.dll
 0000:ffff1000       .debug$S                   10000000     ws2_32:WS2_32.dll
 0000:ffff1000       .debug$S                   10000000     Mswsock:MSWSOCK.dll
 0000:ffff1000       .debug$S                   10000000     kernel32:KERNEL32.dll
 0000:ffff1000       .debug$S                   10000000     kernel32:KERNEL32.dll
 0000:ffff1000       .debug$S                   10000000     kernel32:KERNEL32.dll
 0000:ffff1000       .debug$S                   10000000     kernel32:KERNEL32.dll
 0000:ffff1000       .debug$S                   10000000     kernel32:KERNEL32.dll
 0000:ffff1000       .debug$S                   10000000     kernel32:KERNEL32.dll
 0000:ffff1000       .debug$S                   10000000     kernel32:KERNEL32.dll
 0000:ffff1000       .debug$S                   10000000     kernel32:KERNEL32.dll
 0000:ffff1000       .debug$S                   10000000     kernel32:KERNEL32.dll
 0000:ffff1000       .debug$S                   10000000     kernel32:KERNEL32.dll
 0000:ffff1000       .debug$S                   10000000     kernel32:KERNEL32.dll
 0000:ffff1000       .debug$S                   10000000     kernel32:KERNEL32.dll
 0000:ffff1000       .debug$S                   10000000     kernel32:KERNEL32.dll
 0000:ffff1000       .debug$S                   10000000     kernel32:KERNEL32.dll
 0000:ffff1000       .debug$S                   10000000     kernel32:KERNEL32.dll
 0000:ffff1000       .debug$S                   10000000     kernel32:KERNEL32.dll
 0000:ffff1000       .debug$S                   10000000     kernel32:KERNEL32.dll
 0000:ffff1000       .debug$S                   10000000     kernel32:KERNEL32.dll
 0000:ffff1000       .debug$S                   10000000     kernel32:KERNEL32.dll
 0000:ffff1000       .debug$S                   10000000     kernel32:KERNEL32.dll
 0000:ffff1000       .debug$S                   10000000     kernel32:KERNEL32.dll
 0000:ffff1000       .debug$S                   10000000     kernel32:KERNEL32.dll
 0000:ffff1000       .debug$S                   10000000     kernel32:KERNEL32.dll
 0000:ffff1000       .debug$S                   10000000     kernel32:KERNEL32.dll
 0000:ffff1000       .debug$S                   10000000     kernel32:KERNEL32.dll
 0000:ffff1000       .debug$S                   10000000     kernel32:KERNEL32.dll
 0000:ffff1000       .debug$S                   10000000     kernel32:KERNEL32.dll
 0000:ffff1000       .debug$S                   10000000     kernel32:KERNEL32.dll
 0000:ffff1000       .debug$S                   10000000     kernel32:KERNEL32.dll
 0000:ffff1000       .debug$S                   10000000     kernel32:KERNEL32.dll
 0000:ffff1000       .debug$S                   10000000     kernel32:KERNEL32.dll
 0000:ffff1000       .debug$S                   10000000     kernel32:KERNEL32.dll
 0000:ffff1000       .debug$S                   10000000     kernel32:KERNEL32.dll
 0000:ffff1000       .debug$S                   10000000     kernel32:KERNEL32.dll
 0000:ffff1000       .debug$S                   10000000     kernel32:KERNEL32.dll
 0000:ffff1000       .debug$S                   10000000     kernel32:KERNEL32.dll
 0000:ffff1000       .debug$S                   10000000     kernel32:KERNEL32.dll
 0000:ffff1000       .debug$S                   10000000     kernel32:KERNEL32.dll
 0000:ffff1000       .debug$S                   10000000     kernel32:KERNEL32.dll
 0000:ffff1000       .debug$S                   10000000     kernel32:KERNEL32.dll
 0000:ffff1000       .debug$S                   10000000     kernel32:KERNEL32.dll
 0000:ffff1000       .debug$S                   10000000     kernel32:KERNEL32.dll
 0000:ffff1000       .debug$S                   10000000     kernel32:KERNEL32.dll
 0000:ffff1000       .debug$S                   10000000     kernel32:KERNEL32.dll
 0000:ffff1000       .debug$S                   10000000     kernel32:KERNEL32.dll
 0000:ffff1000       .debug$S                   10000000     kernel32:KERNEL32.dll
 0000:ffff1000       .debug$S                   10000000     kernel32:KERNEL32.dll
 0000:ffff1000       .debug$S                   10000000     kernel32:KERNEL32.dll
 0000:ffff1000       .debug$S                   10000000     kernel32:KERNEL32.dll
 0000:ffff1000       .debug$S                   10000000     kernel32:KERNEL32.dll
 0000:ffff1000       .debug$S                   10000000     kernel32:KERNEL32.dll
 0000:ffff1000       .debug$S                   10000000     kernel32:KERNEL32.dll
 0000:ffff1000       .debug$S                   10000000     kernel32:KERNEL32.dll
 0000:ffff1000       .debug$S                   10000000     kernel32:KERNEL32.dll
 0000:ffff1000       .debug$S                   10000000     kernel32:KERNEL32.dll
 0000:ffff1000       .debug$S                   10000000     kernel32:KERNEL32.dll
 0000:ffff1000       .debug$S                   10000000     kernel32:KERNEL32.dll
 0000:ffff1000       .debug$S                   10000000     kernel32:KERNEL32.dll
 0000:ffff1000       .debug$S                   10000000     kernel32:KERNEL32.dll
 0000:ffff1000       .debug$S                   10000000     kernel32:KERNEL32.dll
 0000:ffff1000       .debug$S                   10000000     kernel32:KERNEL32.dll
 0000:ffff1000       .debug$S                   10000000     kernel32:KERNEL32.dll
 0000:ffff1000       .debug$S                   10000000     kernel32:KERNEL32.dll
 0000:ffff1000       .debug$S                   10000000     kernel32:KERNEL32.dll
 0000:ffff1000       .debug$S                   10000000     kernel32:KERNEL32.dll
 0000:ffff1000       .debug$S                   10000000     kernel32:KERNEL32.dll
 0000:ffff1000       .debug$S                   10000000     kernel32:KERNEL32.dll
 0000:ffff1000       .debug$S                   10000000     kernel32:KERNEL32.dll
 0000:ffff1000       .debug$S                   10000000     kernel32:KERNEL32.dll
 0000:ffff1000       .debug$S                   10000000     kernel32:KERNEL32.dll
 0000:ffff1000       .debug$S                   10000000     vcruntime:VCRUNTIME140.dll
 0000:ffff1000       .debug$S                   10000000     vcruntime:VCRUNTIME140.dll
 0000:ffff1000       .debug$S                   10000000     vcruntime:VCRUNTIME140.dll
 0000:ffff1000       .debug$S                   10000000     ucrt:api-ms-win-crt-heap-l1-1-0.dll
 0000:ffff1000       .debug$S                   10000000     ucrt:api-ms-win-crt-heap-l1-1-0.dll
 0000:ffff1000       .debug$S                   10000000     ucrt:api-ms-win-crt-stdio-l1-1-0.dll
 0000:ffff1000       .debug$S                   10000000     ucrt:api-ms-win-crt-string-l1-1-0.dll
 0000:ffff1000       .debug$S                   10000000     ucrt:api-ms-win-crt-runtime-l1-1-0.dll
 0000:ffff1000       .debug$S                   10000000     ucrt:api-ms-win-crt-runtime-l1-1-0.dll
 0000:ffff1000       .debug$S                   10000000     ucrt:api-ms-win-crt-runtime-l1-1-0.dll
 0000:ffff1000       .debug$S                   10000000     ucrt:api-ms-win-crt-runtime-l1-1-0.dll
 0000:ffff1000       .debug$S                   10000000     ucrt:api-ms-win-crt-runtime-l1-1-0.dll
 0000:ffff1000       .debug$S                   10000000     ucrt:api-ms-win-crt-runtime-l1-1-0.dll
 0000:ffff1000       .debug$S                   10000000     ucrt:api-ms-win-crt-runtime-l1-1-0.dll
 0000:ffff1000       .debug$S                   10000000     ucrt:api-ms-win-crt-runtime-l1-1-0.dll
 0000:ffff1000       .debug$S                   10000000     ucrt:api-ms-win-crt-runtime-l1-1-0.dll
 0000:ffff1000       .debug$S                   10000000     ucrt:api-ms-win-crt-runtime-l1-1-0.dll
 0000:ffff1000       .debug$S                   10000000     ucrt:api-ms-win-crt-runtime-l1-1-0.dll
 0000:ffff1000       .debug$S                   10000000     ucrt:api-ms-win-crt-runtime-l1-1-0.dll
 0000:ffff1000       .debug$S                   10000000     ucrt:api-ms-win-crt-runtime-l1-1-0.dll
 0000:ffff1000       .debug$S                   10000000     nio.exp
 0000:ffff1000       .debug$S                   10000000     ws2_32:WS2_32.dll
 0001:00002204       _setConnectionReset        10003204 f   Net.obj
 0001:0000222b       _setGroupSourceReqOption   1000322b f   Net.obj
 0001:00004602       _throwWindowsException     10005602 f   WindowsNativeDispatcher.obj
 0001:00004a60       $$000000                   10005a60     MSVCRT:lldvrm.obj
 0001:00004b40       $$000000                   10005b40     MSVCRT:lldiv.obj
 0001:00004bf0       $$000000                   10005bf0     MSVCRT:llrem.obj
 0001:00004ca2       ?dllmain_crt_dispatch@@YGHQAUHINSTANCE__@@KQAX@Z 10005ca2 f   MSVCRT:dll_dllmain.obj
 0001:00004cf5       ?dllmain_crt_process_attach@@YAHQAUHINSTANCE__@@QAX@Z 10005cf5 f   MSVCRT:dll_dllmain.obj
 0001:00004dff       ?dllmain_crt_process_detach@@YAH_N@Z 10005dff f   MSVCRT:dll_dllmain.obj
 0001:00004e91       ?dllmain_dispatch@@YAHQAUHINSTANCE__@@KQAX@Z 10005e91 f   MSVCRT:dll_dllmain.obj
 0001:00004f97       ?dllmain_raw@@YGHQAUHINSTANCE__@@KQAX@Z 10005f97 f   MSVCRT:dll_dllmain.obj
 0001:00005106       ___get_entropy             10006106 f   MSVCRT:gs_support.obj
 0001:00005201       ?find_pe_section@@YAPAU_IMAGE_SECTION_HEADER@@QAEI@Z 10006201 f   MSVCRT:utility.obj
 0001:00005680       $$000000                   10006680     MSVCRT:sehprolg4.obj
 0002:00000a90       _GS_ExceptionPointers      10007a90     MSVCRT:gs_report.obj
 0002:00000e48       __sehtable$?dllmain_crt_process_attach@@YAHQAUHINSTANCE__@@QAX@Z 10007e48     MSVCRT:dll_dllmain.obj
 0002:00000e68       __sehtable$?dllmain_crt_process_detach@@YAH_N@Z 10007e68     MSVCRT:dll_dllmain.obj
 0002:00000e88       __sehtable$?dllmain_dispatch@@YAHQAUHINSTANCE__@@KQAX@Z 10007e88     MSVCRT:dll_dllmain.obj
 0002:00000ea8       __sehtable$___scrt_is_nonwritable_in_current_image 10007ea8     MSVCRT:utility.obj
 0002:00000ed0       .edata                     10007ed0     nio.exp
 0002:00000ef8       rgpv                       10007ef8     nio.exp
 0002:000011bc       rgszName                   100081bc     nio.exp
 0002:00001480       rgwOrd                     10008480     nio.exp
 0002:000015e2       szName                     100085e2     nio.exp
 0002:000015ea       $N00001                    100085ea     nio.exp
 0002:000015f8       $N00002                    100085f8     nio.exp
 0002:00001622       $N00003                    10008622     nio.exp
 0002:0000164f       $N00004                    1000864f     nio.exp
 0002:00001678       $N00005                    10008678     nio.exp
 0002:000016ac       $N00006                    100086ac     nio.exp
 0002:000016db       $N00007                    100086db     nio.exp
 0002:0000170c       $N00008                    1000870c     nio.exp
 0002:0000173a       $N00009                    1000873a     nio.exp
 0002:00001767       $N00010                    10008767     nio.exp
 0002:00001795       $N00011                    10008795     nio.exp
 0002:000017c3       $N00012                    100087c3     nio.exp
 0002:000017f2       $N00013                    100087f2     nio.exp
 0002:0000181d       $N00014                    1000881d     nio.exp
 0002:00001846       $N00015                    10008846     nio.exp
 0002:00001876       $N00016                    10008876     nio.exp
 0002:000018a1       $N00017                    100088a1     nio.exp
 0002:000018cf       $N00018                    100088cf     nio.exp
 0002:00001906       $N00019                    10008906     nio.exp
 0002:00001934       $N00020                    10008934     nio.exp
 0002:00001961       $N00021                    10008961     nio.exp
 0002:0000198f       $N00022                    1000898f     nio.exp
 0002:000019be       $N00023                    100089be     nio.exp
 0002:000019eb       $N00024                    100089eb     nio.exp
 0002:00001a19       $N00025                    10008a19     nio.exp
 0002:00001a49       $N00026                    10008a49     nio.exp
 0002:00001a76       $N00027                    10008a76     nio.exp
 0002:00001aa8       $N00028                    10008aa8     nio.exp
 0002:00001ad5       $N00029                    10008ad5     nio.exp
 0002:00001b06       $N00030                    10008b06     nio.exp
 0002:00001b34       $N00031                    10008b34     nio.exp
 0002:00001b63       $N00032                    10008b63     nio.exp
 0002:00001b84       $N00033                    10008b84     nio.exp
 0002:00001ba7       $N00034                    10008ba7     nio.exp
 0002:00001bd4       $N00035                    10008bd4     nio.exp
 0002:00001bf5       $N00036                    10008bf5     nio.exp
 0002:00001c16       $N00037                    10008c16     nio.exp
 0002:00001c38       $N00038                    10008c38     nio.exp
 0002:00001c59       $N00039                    10008c59     nio.exp
 0002:00001c80       $N00040                    10008c80     nio.exp
 0002:00001ca4       $N00041                    10008ca4     nio.exp
 0002:00001cc4       $N00042                    10008cc4     nio.exp
 0002:00001cf4       $N00043                    10008cf4     nio.exp
 0002:00001d1d       $N00044                    10008d1d     nio.exp
 0002:00001d50       $N00045                    10008d50     nio.exp
 0002:00001d70       $N00046                    10008d70     nio.exp
 0002:00001da4       $N00047                    10008da4     nio.exp
 0002:00001dc2       $N00048                    10008dc2     nio.exp
 0002:00001dea       $N00049                    10008dea     nio.exp
 0002:00001e12       $N00050                    10008e12     nio.exp
 0002:00001e45       $N00051                    10008e45     nio.exp
 0002:00001e73       $N00052                    10008e73     nio.exp
 0002:00001e94       $N00053                    10008e94     nio.exp
 0002:00001eba       $N00054                    10008eba     nio.exp
 0002:00001ee0       $N00055                    10008ee0     nio.exp
 0002:00001f06       $N00056                    10008f06     nio.exp
 0002:00001f25       $N00057                    10008f25     nio.exp
 0002:00001f55       $N00058                    10008f55     nio.exp
 0002:00001f7d       $N00059                    10008f7d     nio.exp
 0002:00001faa       $N00060                    10008faa     nio.exp
 0002:00001fce       $N00061                    10008fce     nio.exp
 0002:00001ff2       $N00062                    10008ff2     nio.exp
 0002:00002011       $N00063                    10009011     nio.exp
 0002:0000203a       $N00064                    1000903a     nio.exp
 0002:0000205c       $N00065                    1000905c     nio.exp
 0002:00002079       $N00066                    10009079     nio.exp
 0002:0000209e       $N00067                    1000909e     nio.exp
 0002:000020c2       $N00068                    100090c2     nio.exp
 0002:000020e6       $N00069                    100090e6     nio.exp
 0002:00002109       $N00070                    10009109     nio.exp
 0002:0000212e       $N00071                    1000912e     nio.exp
 0002:00002152       $N00072                    10009152     nio.exp
 0002:0000217c       $N00073                    1000917c     nio.exp
 0002:0000219f       $N00074                    1000919f     nio.exp
 0002:000021c5       $N00075                    100091c5     nio.exp
 0002:000021eb       $N00076                    100091eb     nio.exp
 0002:00002211       $N00077                    10009211     nio.exp
 0002:00002232       $N00078                    10009232     nio.exp
 0002:00002252       $N00079                    10009252     nio.exp
 0002:00002286       $N00080                    10009286     nio.exp
 0002:000022b9       $N00081                    100092b9     nio.exp
 0002:000022ec       $N00082                    100092ec     nio.exp
 0002:0000231f       $N00083                    1000931f     nio.exp
 0002:0000234c       $N00084                    1000934c     nio.exp
 0002:00002384       $N00085                    10009384     nio.exp
 0002:000023b0       $N00086                    100093b0     nio.exp
 0002:000023df       $N00087                    100093df     nio.exp
 0002:0000240a       $N00088                    1000940a     nio.exp
 0002:00002436       $N00089                    10009436     nio.exp
 0002:00002462       $N00090                    10009462     nio.exp
 0002:0000248f       $N00091                    1000948f     nio.exp
 0002:000024cf       $N00092                    100094cf     nio.exp
 0002:0000250f       $N00093                    1000950f     nio.exp
 0002:00002550       $N00094                    10009550     nio.exp
 0002:00002597       $N00095                    10009597     nio.exp
 0002:000025e3       $N00096                    100095e3     nio.exp
 0002:00002629       $N00097                    10009629     nio.exp
 0002:0000267c       $N00098                    1000967c     nio.exp
 0002:000026c2       $N00099                    100096c2     nio.exp
 0002:00002704       $N00100                    10009704     nio.exp
 0002:00002744       $N00101                    10009744     nio.exp
 0002:00002783       $N00102                    10009783     nio.exp
 0002:000027c6       $N00103                    100097c6     nio.exp
 0002:00002814       $N00104                    10009814     nio.exp
 0002:00002854       $N00105                    10009854     nio.exp
 0002:00002893       $N00106                    10009893     nio.exp
 0002:000028cd       $N00107                    100098cd     nio.exp
 0002:00002908       $N00108                    10009908     nio.exp
 0002:00002941       $N00109                    10009941     nio.exp
 0002:0000297f       $N00110                    1000997f     nio.exp
 0002:000029b7       $N00111                    100099b7     nio.exp
 0002:000029f9       $N00112                    100099f9     nio.exp
 0002:00002a3a       $N00113                    10009a3a     nio.exp
 0002:00002a7c       $N00114                    10009a7c     nio.exp
 0002:00002ab1       $N00115                    10009ab1     nio.exp
 0002:00002ae9       $N00116                    10009ae9     nio.exp
 0002:00002b2b       $N00117                    10009b2b     nio.exp
 0002:00002b6e       $N00118                    10009b6e     nio.exp
 0002:00002ba6       $N00119                    10009ba6     nio.exp
 0002:00002be3       $N00120                    10009be3     nio.exp
 0002:00002c1b       $N00121                    10009c1b     nio.exp
 0002:00002c53       $N00122                    10009c53     nio.exp
 0002:00002c8f       $N00123                    10009c8f     nio.exp
 0002:00002cd2       $N00124                    10009cd2     nio.exp
 0002:00002d12       $N00125                    10009d12     nio.exp
 0002:00002d4a       $N00126                    10009d4a     nio.exp
 0002:00002d95       $N00127                    10009d95     nio.exp
 0002:00002dda       $N00128                    10009dda     nio.exp
 0002:00002e17       $N00129                    10009e17     nio.exp
 0002:00002e4d       $N00130                    10009e4d     nio.exp
 0002:00002e88       $N00131                    10009e88     nio.exp
 0002:00002ec3       $N00132                    10009ec3     nio.exp
 0002:00002f00       $N00133                    10009f00     nio.exp
 0002:00002f39       $N00134                    10009f39     nio.exp
 0002:00002f74       $N00135                    10009f74     nio.exp
 0002:00002fae       $N00136                    10009fae     nio.exp
 0002:00002fe1       $N00137                    10009fe1     nio.exp
 0002:00003020       $N00138                    1000a020     nio.exp
 0002:0000305d       $N00139                    1000a05d     nio.exp
 0002:00003099       $N00140                    1000a099     nio.exp
 0002:000030d7       $N00141                    1000a0d7     nio.exp
 0002:00003117       $N00142                    1000a117     nio.exp
 0002:00003151       $N00143                    1000a151     nio.exp
 0002:00003190       $N00144                    1000a190     nio.exp
 0002:000031d1       $N00145                    1000a1d1     nio.exp
 0002:00003218       $N00146                    1000a218     nio.exp
 0002:00003255       $N00147                    1000a255     nio.exp
 0002:0000329a       $N00148                    1000a29a     nio.exp
 0002:000032d7       $N00149                    1000a2d7     nio.exp
 0002:00003310       $N00150                    1000a310     nio.exp
 0002:0000334c       $N00151                    1000a34c     nio.exp
 0002:0000338c       $N00152                    1000a38c     nio.exp
 0002:000033d3       $N00153                    1000a3d3     nio.exp
 0002:00003419       $N00154                    1000a419     nio.exp
 0002:00003460       $N00155                    1000a460     nio.exp
 0002:000034a0       $N00156                    1000a4a0     nio.exp
 0002:000034e2       $N00157                    1000a4e2     nio.exp
 0002:00003521       $N00158                    1000a521     nio.exp
 0002:0000355b       $N00159                    1000a55b     nio.exp
 0002:000035a4       $N00160                    1000a5a4     nio.exp
 0002:000035da       $N00161                    1000a5da     nio.exp
 0002:00003619       $N00162                    1000a619     nio.exp
 0002:00003657       $N00163                    1000a657     nio.exp
 0002:00003699       $N00164                    1000a699     nio.exp
 0002:000036d1       $N00165                    1000a6d1     nio.exp
 0002:0000370e       $N00166                    1000a70e     nio.exp
 0002:0000374a       $N00167                    1000a74a     nio.exp
 0002:00003791       $N00168                    1000a791     nio.exp
 0002:000037d3       $N00169                    1000a7d3     nio.exp
 0002:00003810       $N00170                    1000a810     nio.exp
 0002:00003849       $N00171                    1000a849     nio.exp
 0002:00003888       $N00172                    1000a888     nio.exp
 0002:000038c5       $N00173                    1000a8c5     nio.exp
 0002:000038fd       $N00174                    1000a8fd     nio.exp
 0002:00003943       $N00175                    1000a943     nio.exp
 0002:0000398a       $N00176                    1000a98a     nio.exp
 0002:000039c5       $N00177                    1000a9c5     nio.exp
 0002:00003dba       .idata$6                   1000adba     ws2_32:WS2_32.dll
 0002:00003e9e       .idata$6                   1000ae9e     java:java.dll
 0002:00003fee       .idata$6                   1000afee     net:net.dll
 0002:00004262       .idata$6                   1000b262     advapi32:ADVAPI32.dll
 0002:00004280       .idata$6                   1000b280     Mswsock:MSWSOCK.dll
 0002:000047e4       .idata$6                   1000b7e4     kernel32:KERNEL32.dll
 0002:00004836       .idata$6                   1000b836     vcruntime:VCRUNTIME140.dll
 0002:00004926       .idata$6                   1000b926     ucrt:api-ms-win-crt-heap-l1-1-0.dll
 0002:00004946       .idata$6                   1000b946     ucrt:api-ms-win-crt-stdio-l1-1-0.dll
 0002:00004966       .idata$6                   1000b966     ucrt:api-ms-win-crt-string-l1-1-0.dll
 0002:00004988       .idata$6                   1000b988     ucrt:api-ms-win-crt-runtime-l1-1-0.dll
 0003:00000000       ?loopback_available@?6??Java_sun_nio_ch_Net_socket0@@9@9 1000c000     Net.obj
 0003:00000028       _dci_senderID              1000c028     DatagramChannelImpl.obj
 0003:0000002c       _dci_senderAddrID          1000c02c     DatagramChannelImpl.obj
 0003:00000030       _dci_senderPortID          1000c030     DatagramChannelImpl.obj
 0003:00000034       _isa_class                 1000c034     DatagramChannelImpl.obj
 0003:00000038       _isa_ctorID                1000c038     DatagramChannelImpl.obj
 0003:0000003c       _chan_fd                   1000c03c     FileChannelImpl.obj
 0003:00000040       _key_volumeSN              1000c040     FileKey.obj
 0003:00000044       _key_indexHigh             1000c044     FileKey.obj
 0003:00000048       _key_indexLow              1000c048     FileKey.obj
 0003:0000004c       _handle_fdID               1000c04c     IOUtil.obj
 0003:00000050       _fd_fdID                   1000c050     IOUtil.obj
 0003:00000054       _completionStatus_error    1000c054     Iocp.obj
 0003:00000058       _completionStatus_bytesTransferred 1000c058     Iocp.obj
 0003:0000005c       _completionStatus_completionKey 1000c05c     Iocp.obj
 0003:00000060       _completionStatus_overlapped 1000c060     Iocp.obj
 0003:00000064       ?handle_fdID@?3??Java_java_nio_MappedByteBuffer_force0@@9@9 1000c064     MappedByteBuffer.obj
 0003:00000068       _fd_fdID                   1000c068     ServerSocketChannelImpl.obj
 0003:0000006c       _isa_class                 1000c06c     ServerSocketChannelImpl.obj
 0003:00000070       _isa_ctorID                1000c070     ServerSocketChannelImpl.obj
 0003:00000074       _ia_addrID                 1000c074     SocketChannelImpl.obj
 0003:00000078       _AcceptEx_func             1000c078     WindowsAsynchronousServerSocketChannelImpl.obj
 0003:0000007c       _ConnectEx_func            1000c07c     WindowsAsynchronousSocketChannelImpl.obj
 0003:00000080       _findFirst_handle          1000c080     WindowsNativeDispatcher.obj
 0003:00000084       _findFirst_name            1000c084     WindowsNativeDispatcher.obj
 0003:00000088       _findFirst_attributes      1000c088     WindowsNativeDispatcher.obj
 0003:0000008c       _findStream_handle         1000c08c     WindowsNativeDispatcher.obj
 0003:00000090       _findStream_name           1000c090     WindowsNativeDispatcher.obj
 0003:00000094       _volumeInfo_fsName         1000c094     WindowsNativeDispatcher.obj
 0003:00000098       _volumeInfo_volName        1000c098     WindowsNativeDispatcher.obj
 0003:0000009c       _volumeInfo_volSN          1000c09c     WindowsNativeDispatcher.obj
 0003:000000a0       _volumeInfo_flags          1000c0a0     WindowsNativeDispatcher.obj
 0003:000000a4       _diskSpace_bytesAvailable  1000c0a4     WindowsNativeDispatcher.obj
 0003:000000a8       _diskSpace_totalBytes      1000c0a8     WindowsNativeDispatcher.obj
 0003:000000ac       _diskSpace_totalFree       1000c0ac     WindowsNativeDispatcher.obj
 0003:000000b0       _diskSpace_bytesPerSector  1000c0b0     WindowsNativeDispatcher.obj
 0003:000000b4       _account_domain            1000c0b4     WindowsNativeDispatcher.obj
 0003:000000b8       _account_name              1000c0b8     WindowsNativeDispatcher.obj
 0003:000000bc       _account_use               1000c0bc     WindowsNativeDispatcher.obj
 0003:000000c0       _aclInfo_aceCount          1000c0c0     WindowsNativeDispatcher.obj
 0003:000000c4       _completionStatus_error    1000c0c4     WindowsNativeDispatcher.obj
 0003:000000c8       _completionStatus_bytesTransferred 1000c0c8     WindowsNativeDispatcher.obj
 0003:000000cc       _completionStatus_completionKey 1000c0cc     WindowsNativeDispatcher.obj
 0003:000000d0       ?zerotime@?1??Java_sun_nio_ch_WindowsSelectorImpl_00024SubSelector_poll0@@9@9 1000c0d0     WindowsSelectorImpl.obj
 0003:000000d8       ?__proc_attached@@3HA      1000c0d8     MSVCRT:dll_dllmain.obj
 0003:000000e0       _GS_ExceptionRecord        1000c0e0     MSVCRT:gs_report.obj
 0003:00000130       _GS_ContextRecord          1000c130     MSVCRT:gs_report.obj
 0003:00000420       ?is_initialized_as_dll@@3_NA 1000c420     MSVCRT:utility.obj
 0003:00000421       ?module_local_atexit_table_initialized@@3_NA 1000c421     MSVCRT:utility.obj
 0003:00000424       ?module_local_atexit_table@@3U_onexit_table_t@@A 1000c424     MSVCRT:utility.obj
 0003:00000430       ?module_local_at_quick_exit_table@@3U_onexit_table_t@@A 1000c430     MSVCRT:utility.obj
 0004:00000060       $R000000                   1000d060     nio.dll.res
